:100000000C9489070C94AF070C94AF070C94AF07BE
:100010000C94AF070C94AF070C94AF070C94AF0788
:100020000C94AF070C94AF070C9418090C94340986
:100030000C94AF070C94AF070C94AF070C94AF0768
:100040000C94AF070C94AF070C94AF070C94AF0758
:100050000C94AF070C94AF070C94AF070C94AF0748
:100060000C94AF070C94AF070C94AF070C94AF0738
:100070000C94AF070C94AF070C94AF070C94AF0728
:100080000C94AF070C94AF070C94AF070C94AF0718
:100090000C94AF070C94AF070C94AF070C94BF0AF5
:1000A0000C94FC0A0C94390B0C94760B0C94AF074F
:1000B0000C94AF070C94AF070C94AF070C94AF07E8
:1000C0000C94AF070C94AF070C94AF070C94AF07D8
:1000D0000C94AF070C94AF070C94AF070C94AF07C8
:1000E0000C94AF070C94AF070C94AF070C94AF07B8
:1000F0000C94AF070C94AF070C94AF070C94AF07A8
:100100000C94AF070C94AF070C94AF070C94AF0797
:100110000C94AF070C94AF070C94AF070C94CB0969
:100120000C94080A0C94450A0C94820A0C94AF07AC
:100130000C94AF070C94AF070C94AF070C94AF0767
:100140000C94AF070C94AF070C94AF070C94AF0757
:100150000C94AF070C94AF070C94AF070C94AF0747
:100160000C94AF070C94AF070C94AF070C94AF0737
:100170000C94AF070C94AF070C94AF070C94AF0727
:100180000C94AF070C94AF070C94AF070C94AF0717
:100190000C94AF070C94AF070C94AF070C94AF0707
:1001A0000C94AF070C94AF070C94AF070C94AF07F7
:1001B0000C94AF070C94AF070C94AF070C94AF07E7
:1001C0000C94AF070C94AF070C94AF070C94AF07D7
:1001D0000C94AF070C94AF070C94AF070C94AF07C7
:1001E0000C94AF070C94AF070C94AF070C94AF07B7
:1001F0000C94AF071F1E1C1E191E161E131E101E68
:100200000D1E0A1E071E041E011EFE1DFB1DF81DED
:10021000F51DF21DEF1DEC1DE91DE61DE01DE31DA2
:100220003C696E70757420747970653D22737562D7
:100230006D697422207374796C653D226865696705
:1002400068743A203530707822206E616D653D22E9
:10025000746F67676C65222076616C75653D224C12
:10026000454434222F3E266E627370266E62737090
:100270003C696E70757420747970653D2273756287
:100280006D697422207374796C653D2268656967B5
:1002900068743A203530707822206E616D653D2299
:1002A000746F67676C65222076616C75653D224CC2
:1002B000454435222F3E266E627370266E6273703F
:1002C0003C696E70757420747970653D2273756237
:1002D0006D697422207374796C653D226865696765
:1002E00068743A203530707822206E616D653D2249
:1002F000746F67676C65222076616C75653D224C72
:10030000454436222F3E266E627370266E627370ED
:100310003C696E70757420747970653D22737562E6
:100320006D697422207374796C653D226865696714
:1003300068743A203530707822206E616D653D22F8
:10034000746F67676C65222076616C75653D224C21
:10035000454437222F3E266E627370266E6273709C
:100360003C2F6669656C647365743E3C2F666F72E2
:100370006D3E3C2F74643E3C74643E266E62737026
:100380003B3C2F74643E3C2F74723E3C2F74616280
:100390006C653E3C2F74643E3C74642077696474E1
:1003A000683D323025253E3C2F74643E3C2F7472EC
:1003B0003E3C2F7461626C653E3C2F626F64793EF7
:1003C0003C2F68746D6C3E003C74723E3C74643E1D
:1003D0003C666F726D206D6574686F643D22676561
:1003E00074223E3C696E70757420747970653D228C
:1003F0007375626D697422207374796C653D22682F
:1004000065696768743A2035307078222076616CAF
:1004100075653D2252656672657368222F3E3C2FDA
:10042000666F726D3E3C2F74643E3C2F74723E3C8E
:100430002F7461626C653E3C62723E3C666F726D09
:100440002069643D22666F726D226E616D653D228A
:10045000666F726D22206D6574686F643D226765FA
:10046000742220616374696F6E3D22696E646578E1
:100470002E68746D6C223E3C6669656C64736574AD
:10048000207374796C653D2277696474683A20330F
:1004900030303B223E3C6C6567656E643E4C4544A3
:1004A00020636F6E74726F6C3C2F6C6567656E6451
:1004B0003E3C696E70757420747970653D22737569
:1004C000626D697422207374796C653D2268656978
:1004D0006768743A203530707822206E616D653D12
:1004E00022746F67676C65222076616C75653D22AA
:1004F0004C454430222F3E266E627370266E627326
:10050000703C696E70757420747970653D227375E6
:10051000626D697422207374796C653D2268656927
:100520006768743A203530707822206E616D653DC1
:1005300022746F67676C65222076616C75653D2259
:100540004C454431222F3E266E627370266E6273D4
:10055000703C696E70757420747970653D22737596
:10056000626D697422207374796C653D22686569D7
:100570006768743A203530707822206E616D653D71
:1005800022746F67676C65222076616C75653D2209
:100590004C454432222F3E266E627370266E627383
:1005A000703C696E70757420747970653D22737546
:1005B000626D697422207374796C653D2268656987
:1005C0006768743A203530707822206E616D653D21
:1005D00022746F67676C65222076616C75653D22B9
:1005E0004C454433222F3E266E627370266E627332
:1005F000703C703E003C2F74643E3C74643E3C6230
:100600003E3C2F623E3C2F74643E3C2F74723E0091
:100610003C74723E3C74643E54656D7065726174E6
:100620007572653A20003C2F74643E3C74643E3C15
:10063000623E3C2F623E3C2F74643E3C2F74723EFF
:10064000003C74723E3C74643E4D414320416464FE
:10065000726573733A20003C2F74643E3C74643EB0
:100660003C623E3C2F623E3C2F74643E3C2F7472D1
:100670003E003C74723E3C74643E495020416464C8
:10068000726573733A2000485454502F312E302035
:10069000323030204F4B0A5365727665723A2077BC
:1006A0006C705F68747470640A436F6E74656E7406
:1006B0002D747970653A20746578742F68746D6C48
:1006C0000A0A3C21444F43545950452048544D4C4C
:1006D000205055424C494320222D2F2F5733432F72
:1006E0002F4454442048544D4C20342E3031204661
:1006F00072616D657365742F2F454E2220226874D8
:1007000074703A2F2F7777772E77332E6F72672F8B
:1007100054522F68746D6C342F6672616D65736509
:10072000742E647464223E3C68746D6C3E3C686553
:1007300061643E3C7469746C653E6F574C2070690F
:10074000636F204854545020576562207365727659
:1007500065723C2F7469746C653E3C2F68656164FA
:100760003E3C626F6479207374796C653D666F6E90
:10077000742D66616D696C793A617269616C3E3C99
:100780007461626C653E3C74723E3C7464207769AF
:100790006474683D3130303E3C2F74643E3C746478
:1007A0003E3C7461626C653E3C74722076616C699B
:1007B000676E3D22746F70223E3C746420776974CA
:1007C000683E3C696D67207372633D226C6F676F92
:1007D0002E6769662220626F726465723D22302244
:1007E00020616C743D226C6F676F227469746C6554
:1007F0003D226C6F676F223E3C2F74643E3C2F7429
:10080000723E3C74723E3C74642077696474683D47
:1008100022353030223E3C68323E576562205365B7
:10082000727665722072756E6E696E67206F6E20CB
:100830006F574C207069636F3C2F68323E3C703EAE
:100840005468652077656220706167652069732050
:1008500073657276656420627920776C705F687466
:10086000747064207573696E6720746865205350D6
:100870004238303020574C414E206D6F64756C65A6
:1008800020616E6420746865206F574C2D70696319
:100890006F26636F70793B20536F66747761726562
:1008A000204150493B206120756E69717565205764
:1008B000692D466920736F6C7574696F6E2066725E
:1008C0006F6D203C623E48264420576972656C6516
:1008D00073732041423C2F623E2E3C2F703E3C6899
:1008E000723E3C7461626C653E004749463839612E
:1008F00045017B00A10000FFFFFF0066990000009A
:10090000FFFFFF21FE114372656174656420776902
:1009100074682047494D50002C0000000045017BC1
:10092000000002FE848FA9CBED0FA39CB4DA8BB339
:10093000DEBCFB0F86E24896E689A6EACAB6EE0B55
:10094000C7F24CD7F68DE7FACEF7FE0F0C0A87C434
:10095000A2F1884C2A97CCA6F3098D4AA7D4AAF510
:100960008A6505B6DCAEF70B0E8BC76471F60C2DED
:10097000ABD7EC36190D3FBAE7F4FA3B8EFFD9F747
:100980007C7BFE9FD32738C80668384398A8187622
:10099000D8D8B2081919E048792279A958A929822A
:1009A000D929B809DAE139CA176A8A419A4A77CA55
:1009B0003AA1FAEAD62AEB005BAB368BAB60BB6B95
:1009C00096EB0BC01BECF5EB2B6CBC458C7B6C9C4D
:1009D0003CBB2CDC2CFB1C1CDD3ACD5BCD7ABD9BDB
:1009E0007DBA6DDB6DFA5D1B1E3A0E5B0E7AFE9AC8
:1009F000BEB9AEDAAEF99E1A5F394F5A4F793F9AB7
:100A0000EFB8EFD9AFD1BF4E010F0DC454D0D0C154
:100A10004B09012D94D4F0CFC34811F34C845411E9
:100A2000CF1DFE5D601A8CF158A6421B04024A9A43
:100A300014B0E0E4C9942A511E68290366B88D09F0
:100A40001831B0F980A6AB5B2465F6F4F9122800E2
:100A5000A12D8836D3790027C761123E5EE0195474
:100A6000A5829625A70A35BA022B31A40694D6642E
:100A7000DAB4D7539D5413503569F6AAD4185A7F67
:100A80007105D6F126D8B07151398DBAF26759BDCA
:100A900068F9BA84D1B6D8DDAF5F4072913B69691D
:100AA000E10C64D59E4DBB7647E05C6FBD22987B20
:100AB000199962CC490FD3128BB7AF81B355FDFAA8
:100AC00098AC6C70E6C50B58AFDECCB96B6CD996A0
:100AD000F70E255DFA76E4D07F47FBCCCB12788306
:100AE000C9A879E77EF0B847E5BAB05B2726CC7C89
:100AF0007517C4D17503C79DDB366FC82B8962EFAC
:100B0000CDFD7878ED56B10FFFCEE3ADC8D9CE411B
:100B10004BF7DCDEB5EFC8E8E70BB72FBE2CD0EF04
:100B2000F7FEF183F78F5B70FC95376020AAD9C57B
:100B3000DE7BD5D1361D75B1FD661E8004E65720DB
:100B400080018E2760851692365E8438A847C18260
:100B5000D0B9D7197B245A87964C2AEEB69D5FDA16
:100B6000F1C7228AFFC1789F63C2D9289A0D20EE6F
:100B7000045F4E21C5D7E3880D7628A37F32FE5748
:100B8000A48B10C6481E8EE21D69DA04C5DDB023B1
:100B90005DCF41009F8822C2B5A07E6BC1449E916B
:100BA0004A228995931866D85B98E7C5E843951162
:100BB0000489E0950ACA39A7661DDAA6618BC621A9
:100BC00079248C51EE59619E63F6F7E1810C0EB9E0
:100BD0001407B36D79629F377A78E69E0CD0B81F00
:100BE0008B94EE46239A1CEAB09C7C9921C6239DE7
:100BF00087DA091B9C1BE658DF84E0A9792AA44EFA
:100C0000663A289BB016DAA8659D01F926A2733AC8
:100C1000385BAA8EE6F8A784935E8AAAA5C43EF93B
:100C2000FE2BA1C9024B43A7268AEAA990BC1A262B
:100C300022A4AD0E5BA356AC3A60A6079B22F76DCB
:100C40000DCEEAFA2990A46E469D8FB69EAA2A9BE5
:100C5000491AB7A6B2DC1AEB6E0653BEABA3A15C71
:100C60003E6B188F1BE8FB6BBBCCEA29ACA6AB76BE
:100C70002BA98B146CABAA81B5322A2A63115BB9FC
:100C8000E58583C64B61BDCB7AC724B109EB991CBE
:100C9000C1E2EABB2E971E984A71C521DFC927BE63
:100CA00050622C28C794B21CAEC7B4AE5B32B916E2
:100CB000E89CAB7AE18E093391F3FAD9B0C02BB737
:100CC000FAAAC554920C31CAEDBD37D68FD8BAFBFB
:100CD00073B02F83AB74A4460F0C28D5828EFC70A2
:100CE000B4A34EBC6F8309960AF0D59A0E0D2CC39F
:100CF00045B38DACD0111C0D73CBF95E9448467191
:100D0000E09D89DE68F09DB7DF67004E88E08313C1
:100D1000FE89E158209EB8E25630DE87E35740ADA9
:100D20005E8AE45550BE87E597635E87E65470DEC1
:100D3000B9E75280BE8AE851903E87E9A7A33E9268
:100D4000EA4FB0DEBAEB4DC05E88ECB3D30E95ED42
:100D50004AE09EBBEE48F02EB5EFBF039FB6F040D1
:100D6000105FBCF16D225FB2F27A30BFA5F3CB43C6
:100D70007FB6F43B505FBDF59C62EFB4F6CA714F8D
:100D8000B6F7D7832F3E11E4976F3EF6E8A74FFDE5
:100D9000FAEC23EF7E11CCC72F3FF1F41B01FCFDD1
:100DA000C3B3AE7F12A4F77F3BC601F0730719A04F
:100DB000010F88C0042A70810C6CA0031F08C108B1
:100DC0004A708214ACA0052F8841CD1500003B4825
:100DD0005454502F312E3020323030204F4B0A5394
:100DE00065727665723A20776C705F6874747064AF
:100DF0000A436F6E74656E742D747970653A20695C
:100E00006D6167652F6769660A0A00485454502F60
:100E1000312E30203430342046696C65206E6F747A
:100E200020666F756E640A5365727665723A207734
:100E30006C705F68747470640A436F6E74656E746E
:100E40002D747970653A20746578742F68746D6CB0
:100E50000A0A3C68746D6C3E3C686561643E3C7493
:100E600069746C653E6F574C207069636F204854FD
:100E7000545020576562207365727665723C2F74FA
:100E800069746C653E3C2F686561643E3C626F64CA
:100E9000793E3C68323E343034202D205061676505
:100EA000206E6F7420666F756E643C2F68323E3C16
:100EB000703E536F7272792C207468652070616780
:100EC0006520796F75206172652072657175657333
:100ED00074696E6720776173206E6F7420666F751A
:100EE0006E64206F6E207468697320736572766516
:100EF000722E3C2F703E3C2F626F64793E3C2F680F
:100F0000746D6C3E006364696E6F70737578585BC6
:100F1000000011241FBECFEFDFE3DEBFCDBF00E036
:100F20000CBF18BE19BE1ABE1BBE1EE2A0E0B0E286
:100F3000E2E8F8E900E00BBF02C007900D92AE387E
:100F4000B107D9F71BBE1EE2AEE8BEE201C01D929A
:100F5000A53DB107E1F70E94723F0C943F4C0C9401
:100F600000009BB78BBFFB018091CA014093CA016F
:100F70007DE970933400E8958093CA019BBF089582
:100F80002091CF0127FDFCCF9BB78BBFFB01809148
:100F9000CA0123E22093CA010A01E8951124809333
:100FA000CA019BBF0895FC019FB7F894E059FF4F19
:100FB00060958081862380839FBF0895FC019FB741
:100FC000F894E059FF4F8081862B80839FBF08955E
:100FD000E0E7F0E08FEF8193E737F105E1F79FB7A6
:100FE000F894809150008260809350009FBF809160
:100FF000510081FFFCCF80E490E061E00E94C509D0
:101000009FB7F894809150008E7F809350009FBFCF
:101010000895282FAB0186958695869590E0C09619
:10102000277061E070E002C0660F771F2A95E2F733
:1010300025E0880F991F2A95E1F70E9485080895F9
:1010400080E260E073E00E94090881E260E073E002
:101050000E94090882E260E073E00E94090883E2CE
:1010600060E073E00E94090884E260E073E00E949F
:10107000090885E260E073E00E94090886E260E00A
:1010800073E00E94090887E260E073E00E940908AB
:1010900088E268E170E00E94090889E268E170E096
:1010A0000E9409088AE268E170E00E9409088BE268
:1010B00068E170E00E9409088CE268E170E00E943B
:1010C00009088DE268E170E00E9409088EE268E19B
:1010D00070E00E9409088FE268E170E00E94090850
:1010E00083E160E073E00E94090882E160E070E063
:1010F0000E9409088BE160E073E00E9409088AE120
:1011000060E070E00E9409080895CF93DF93DC014E
:10111000FC0120E030E0C62FD0E0CE01022E02C05C
:10112000959587950A94E2F780FD408B2F5F3F4F9E
:1011300031962830310589F750FF0CC051FF04C0AB
:1011400015966C93159703C016966C931697119687
:101150006C9302C012966C93DF91CF9108959B011E
:10116000AC01109200048091010480FDFCCFE0E00E
:10117000F4E020873187CA01AA27BB278093B42EC9
:101180009093B52E87E08093000408959FB7F8945C
:101190002091B42E3091B52E60910804709109040D
:1011A0006115710531F48091030480FF02C02F5F47
:1011B0003F4F9FBF40E050E0A90133272227CB01DA
:1011C000A0E0B0E0282B392B4A2B5B2BB901CA01D8
:1011D00008959B01AC0181E0E0E0F4E0828380911E
:1011E000010480FDFCCFE0E0F4E024873587209304
:1011F000B82E3093B92ECA01AA27BB278093B62EEA
:101200009093B72E8091010480FDFCCF85E0E0E053
:10121000F4E082830895E0E0F4E08281869586958B
:101220008095817008958093BA2E9093BB2E089577
:101230001F920F920FB60F9208B60F9218BE11248C
:101240008F939F938091B42E9091B52E01968093A9
:10125000B42E9093B52E9F918F910F9008BE0F9052
:101260000FBE0F901F9018951F920F920FB60F92FE
:1012700008B60F9218BE09B60F9219BE0BB60F92A0
:101280001BBE1124EF92FF920F931F932F933F9356
:101290004F935F936F937F938F939F93AF93BF937E
:1012A000EF93FF932091B42E3091B52E6091B62E1E
:1012B0007091B72E26173707C0F181E0E0E0F4E027
:1012C0008283E091BA2EF091BB2E309771F180911C
:1012D00008049091090440E050E08901FF24EE24C5
:1012E000A0E0B0E0E82AF92A0A2B1B2BCB01A0E0F2
:1012F000B0E0AC01332722278091B82E9091B92E0F
:10130000A0E0B0E0282B392B4A2B5B2B2E153F0594
:101310004007510738F079018A010894E11CF11C5B
:10132000011D111DC801B7011995FF91EF91BF91E2
:10133000AF919F918F917F916F915F914F913F916D
:101340002F911F910F91FF90EF900F900BBE0F9078
:1013500009BE0F9008BE0F900FBE0F901F901895FA
:1013600080E090E064E00E94D30721E0E0E4F0E058
:101370002383E0E0F4E08FEF9FEF8287938710866E
:101380001186228387E0808308951BBEFC0128ED2F
:1013900024BF608308951F920F920FB60F9208B674
:1013A0000F9218BE09B60F9219BE0BB60F921BBE54
:1013B00011242F933F934F935F936F937F938F935A
:1013C0009F93AF93BF93EF93FF93E0E2F2E04481EA
:1013D0005581E091912EF091922E80E092E060E0B4
:1013E0001995FF91EF91BF91AF919F918F917F914F
:1013F0006F915F914F913F912F910F900BBE0F9086
:1014000009BE0F9008BE0F900FBE0F901F90189549
:101410001F920F920FB60F9208B60F9218BE09B620
:101420000F9219BE0BB60F921BBE11242F933F9340
:101430004F935F936F937F938F939F93AF93BF93DC
:10144000EF93FF93E8E2F2E044815581E091912E21
:10145000F091922E80E092E061E01995FF91EF917A
:10146000BF91AF919F918F917F916F915F914F91BC
:101470003F912F910F900BBE0F9009BE0F9008BEA9
:101480000F900FBE0F901F9018951F920F920FB6DE
:101490000F9208B60F9218BE09B60F9219BE0BB67E
:1014A0000F921BBE11242F933F934F935F936F9323
:1014B0007F938F939F93AF93BF93EF93FF93E0E35B
:1014C000F2E044815581E091912EF091922E80E0DE
:1014D00092E062E01995FF91EF91BF91AF919F91DA
:1014E0008F917F916F915F914F913F912F910F90CD
:1014F0000BBE0F9009BE0F9008BE0F900FBE0F904D
:101500001F9018951F920F920FB60F9208B60F9268
:1015100018BE09B60F9219BE0BB60F921BBE11244E
:101520002F933F934F935F936F937F938F939F93EB
:10153000AF93BF93EF93FF93E8E3F2E044815581CB
:10154000E091912EF091922E80E092E063E0199567
:10155000FF91EF91BF91AF919F918F917F916F918B
:101560005F914F913F912F910F900BBE0F9009BE4D
:101570000F9008BE0F900FBE0F901F9018951F92EE
:101580000F920FB60F9208B60F9218BE09B60F92BF
:1015900019BE0BB60F921BBE11242F933F934F938E
:1015A0005F936F937F938F939F93AF93BF93EF93CB
:1015B000FF93E0E6F2E044815581E091942EF091B2
:1015C000952E80E492E060E01995FF91EF91BF9134
:1015D000AF919F918F917F916F915F914F913F91CB
:1015E0002F910F900BBE0F9009BE0F9008BE0F9069
:1015F0000FBE0F901F9018951F920F920FB60F926B
:1016000008B60F9218BE09B60F9219BE0BB60F920C
:101610001BBE11242F933F934F935F936F937F9340
:101620008F939F93AF93BF93EF93FF93E8E6F2E01E
:1016300044815581E091942EF091952E80E492E0C2
:1016400061E01995FF91EF91BF91AF919F918F91BB
:101650007F916F915F914F913F912F910F900BBEB2
:101660000F9009BE0F9008BE0F900FBE0F901F90F5
:1016700018951F920F920FB60F9208B60F9218BED0
:1016800009B60F9219BE0BB60F921BBE11242F93F1
:101690003F934F935F936F937F938F939F93AF93FA
:1016A000BF93EF93FF93E0E7F2E044815581E0912F
:1016B000942EF091952E80E492E062E01995FF91CE
:1016C000EF91BF91AF919F918F917F916F915F91BA
:1016D0004F913F912F910F900BBE0F9009BE0F902D
:1016E00008BE0F900FBE0F901F9018951F920F927B
:1016F0000FB60F9208B60F9218BE09B60F9219BE18
:101700000BB60F921BBE11242F933F934F935F9301
:101710006F937F938F939F93AF93BF93EF93FF93B9
:10172000E8E7F2E044815581E091942EF091952E06
:1017300080E492E063E01995FF91EF91BF91AF9142
:101740009F918F917F916F915F914F913F912F91D9
:101750000F900BBE0F9009BE0F9008BE0F900FBEEA
:101760000F901F90189522E08030920731F48091FD
:10177000902E882359F081E008958054924011F012
:1017800080E008958091932E811181E008952FB714
:10179000F89432E08030930729F46093912E70938F
:1017A000922E07C08054924021F46093942E70933F
:1017B000952E2FBF089522E08030920769F4809122
:1017C000902E8F5F8093902E8150A9F481E090E05D
:1017D00062E00E94D30708958054924061F48091A2
:1017E000932E8F5F8093932E815029F482E090E0B6
:1017F00062E00E94D3070895FF920F931F938C011C
:10180000FFB6F8940E94DB0BF80180818160808331
:10181000FFBE1F910F91FF90089522E08030920744
:1018200069F48091902E81508093902E8823A9F4A2
:1018300081E090E062E00E94DE07089580549240CB
:1018400061F48091932E81508093932E882329F404
:1018500082E090E062E00E94DE070895DF92EF925E
:10186000FF920F931F93CF93DF938C017A01005E59
:101870001F4FC62FD0E083E0CC0FDD1F8A95E1F724
:10188000C00FD11F00521040DFB6F894C8010E946B
:10189000DB0B8881F70180838A8182838981818340
:1018A000C8010E940D0CDFBEDF91CF911F910F91F7
:1018B000FF90EF90DF900895DF92EF92FF920F93E9
:1018C0001F93CF93DF938C017A01005E1F4FC62FC9
:1018D000D0E093E0CC0FDD1F9A95E1F7C00FD11F48
:1018E00000521040DFB6F894C8010E94DB0BF701EC
:1018F0008081888382818A8381818983C8010E9453
:101900000D0CDFBEDF91CF911F910F91FF90EF90F3
:10191000DF900895DF92EF92FF920F931F938C0157
:101920007B01DFB6F8940E94DB0BF8018081807C9C
:10193000F7018083F801808D918DF701858396836F
:10194000F8018281F7018283F8018481F7018483A1
:10195000F8018381F7018383F8018181F701818395
:10196000C8010E940D0CDFBE1F910F91FF90EF90F8
:10197000DF9008951F93FC011FB7F89480818E7F3C
:101980008083CF010E940D0C1FBF1F9108950F93FC
:101990001F938130910589F08130910528F00297DD
:1019A000A9F020E030E020C082E061E20E949022B5
:1019B000182F00E082E060E211C082E065E20E9440
:1019C0009022182F00E082E064E208C082E06FE21B
:1019D0000E949022182F00E082E06EE20E94902286
:1019E000282F30E0202B312BC9011F910F91089532
:1019F000CF92DF92EF92FF921F93CF93DF93EC0190
:101A00007B0182E0C030D80719F480E090E006C086
:101A1000E2E0C034DE0721F581E090E00E94C70CCF
:101A20006C011FB7F894CE010E94DB0B288182E085
:101A30008883CC86DD86F70185819681888F998F92
:101A400082818A8384818C8383818B838181898352
:101A500021708081282B2883CE010E940D0C1FBF8E
:101A6000DF91CF911F91FF90EF90DF90CF9008957D
:101A7000E091962EF091972E8783908761877287E9
:101A80000895E091962EF091972E8387948765872D
:101A9000768708959C01E091982EF091992E08C0C8
:101AA000808191818217930741F00380F481E02DBA
:101AB0003097B1F72EEF3FEF06C0678370874387FB
:101AC000548720E030E0C90108959C01E091982EF0
:101AD000F091992E08C0808191818217930741F07F
:101AE0000380F481E02D3097B1F72EEF3FEF06C071
:101AF000618772874587568720E030E0C9010895E5
:101B0000AF92BF92CF92DF92EF92FF920F931F930B
:101B1000DF93CF930F920F92CDB7DEB76C01162FE4
:101B2000072F7A0159011F5F19831150E091962EFA
:101B3000F091972E2281338184819581BE016F5F60
:101B40007F4F41E050E0F9011995E091962EF09118
:101B5000972E2081318184819581BE016E5F7F4FF8
:101B600041E050E0F90119959A818981981719F09F
:101B700020EF3FEF23C0E091962EF091972E228127
:101B8000338184819581B601412F502FF901199538
:101B9000E091962EF091972E20813181848195815C
:101BA000B701A501F9011995F701808191810E9482
:101BB000EA15F7018083918320E030E0C9010F909E
:101BC0000F90CF91DF911F910F91FF90EF90DF90D9
:101BD000CF90BF90AF9008952F923F924F925F9217
:101BE0006F927F928F929F92AF92BF92CF92DF922D
:101BF000EF92FF920F931F93DF93CF93CDB7DEB792
:101C00006997CDBFDEBF5C014B013A012901170185
:101C1000760189E08983CE01019661E070E0AE0132
:101C20004E5F5F4F28E130E00E94800D9C0197FDE0
:101C300052C0A114B10449F08E819F81A885B98555
:101C4000F50180839183A283B3838114910449F0C9
:101C50008A859B85AC85BD85F40180839183A283B1
:101C6000B3836114710449F08E859F85A889B98971
:101C7000F30180839183A283B3834114510449F01B
:101C80008A899B89AC89BD89F20180839183A28373
:101C9000B3830115110539F08D81992787FD909542
:101CA000F80180839183E114F10439F08C81992744
:101CB00087FD9095F701808391832114310449F0C9
:101CC0008E899F89A88DB98DF10180839183A2832C
:101CD000B3832A813B81C9016996CDBFDEBFCF9115
:101CE000DF911F910F91FF90EF90DF90CF90BF9009
:101CF000AF909F908F907F906F905F904F903F90AC
:101D00002F900895CF92DF92EF92FF920F931F933F
:101D10008C0180E090E060E070E040E050E020E086
:101D200030E0EE24FF24CC24DD240E94EC0D1F9132
:101D30000F91FF90EF90DF90CF900895CF92DF92B8
:101D4000EF92FF920F931F9300E010E0EE24FF2428
:101D5000CC24DD240E94EC0D1F910F91FF90EF9099
:101D6000DF90CF9008950F93DF93CF93CDB7DEB779
:101D70006697CDBFDEBFFC0188E08B83309749F0CA
:101D800080819181A281B3818F839887A987BA8747
:101D900004C01F82188619861A866115710551F0D4
:101DA000FB0180819181A281B3818B879C87AD8764
:101DB000BE8704C01B861C861D861E8641155105E4
:101DC00051F0FA0180819181A281B3818F87988B34
:101DD000A98BBA8B04C01F86188A198A1A8A211502
:101DE000310551F0F90180819181A281B3818B8B02
:101DF0009C8BAD8BBE8B04C01B8A1C8A1D8A1E8ADD
:101E00000E83CE01039664E170E0AE014F5F5F4F39
:101E100022E030E00E94800D9C0197FD02C02981E4
:101E20003A81C9016696CDBFDEBFCF91DF910F9198
:101E300008950F931F938C0180E090E060E070E0C4
:101E400040E050E020E030E00E94B30E1F910F917F
:101E500008950F931F9300E010E00E94B30E1F91AE
:101E60000F910895DF93CF9300D0CDB7DEB784E014
:101E70008983CE01019661E070E0AE014E5F5F4F55
:101E800022E030E00E94800D9C0197FD02C02A8173
:101E90003B81C9012396CDBFDEBFCF91DF9108956D
:101EA0000F931F93DF93CF93CDB7DEB72C97CDBFA2
:101EB000DEBF8B0125E129830E94E6158B839C837D
:101EC000CE01019664E070E0AE014B5F5F4F28E009
:101ED00030E00E94800D9C0197FD0DC02D813E8158
:101EE00037FD09C089859A85AB85BC85F80180835B
:101EF0009183A283B383C9012C96CDBFDEBFCF915E
:101F0000DF911F910F910895AF92BF92CF92DF9210
:101F1000EF92FF920F931F93DF93CF93CDB7DEB76E
:101F20002E97CDBFDEBF5B016A01790122E12B83D1
:101F30000E94E6158D839E83C6010E94E6158F835D
:101F40009887F70180819181A281B3818B879C87DB
:101F5000AD87BE87C8010E94E61589879A87CE01A2
:101F600003966CE070E0AE014F5F5F4F22E030E01F
:101F70000E94800DAC0197FD16C049815A8157FD22
:101F800012C0C416D5061CF440EF5FEF0CC0E09100
:101F9000962EF091972E2281338184819581B5010F
:101FA000F9011995AC01CA012E96CDBFDEBFCF91C4
:101FB000DF911F910F91FF90EF90DF90CF90BF9036
:101FC000AF900895EF92FF920F931F93DF93CF93FB
:101FD000CDB7DEB72897CDBFDEBF7B018A0121E1F7
:101FE0002B830E94E6158D839E83C8010E94E6150F
:101FF0008F839887CE01039666E070E0AE014F5F55
:102000005F4F22E030E00E94800DAC0197FD16C0CA
:1020100049815A8157FD12C0041715071CF440EF7F
:102020005FEF0CC0E091962EF091972E22813381C4
:1020300084819581B701F9011995AC01CA012896EF
:10204000CDBFDEBFCF91DF911F910F91FF90EF9039
:102050000895EF92FF920F931F93DF93CF93CDB725
:10206000DEB72897CDBFDEBF7B018A0120E12B833D
:102070000E94E6158D839E83C8010E94E6158F831A
:102080009887CE01039666E070E0AE014F5F5F4F28
:1020900022E030E00E94800DAC0197FD16C049811E
:1020A0005A8157FD12C0041715071CF440EF5FEF6B
:1020B0000CC0E091962EF091972E20813181848181
:1020C0009581B701F9011995AC01CA012896CDBFD8
:1020D000DEBFCF91DF911F910F91FF90EF90089598
:1020E000EF92FF920F931F93DF93CF93CDB7DEB79D
:1020F0002C97CDBFDEBF9C018B017A01E091982E19
:10210000F091992E08C0808191818217930741F048
:102110000380F481E02D3097B1F72EEF3FEF25C01B
:102120008EE08B83C9010E94E6158D839E83F801A2
:1021300080819181A281B3818F839887A987BA8793
:10214000C7010E94E6158B879C87CE0103966AE043
:1021500070E0AE014F5F5F4F22E030E00E94800DE3
:102160009C0197FD02C029813A81C9012C96CDBFFF
:10217000DEBFCF91DF911F910F91FF90EF900895F7
:102180001F93DF93CF9300D000D0CDB7DEB7DC0133
:10219000162FE091982EF091992E08C080819181A0
:1021A0008A179B0741F00380F481E02D3097B1F747
:1021B0002EEF3FEF1CC045835683238734878DE085
:1021C0008B83CD010E94E6158D839E831C83CE01F7
:1021D000039664E070E0AE014F5F5F4F22E030E0B5
:1021E0000E94800D9C0197FD02C029813A81C9019E
:1021F0002696CDBFDEBFCF91DF911F910895EF925C
:10220000FF920F931F93DF93CF93CDB7DEB72C9739
:10221000CDBFDEBF8B017A012CE02B830E94E61537
:102220008D839E83F80180819181A281B3818F8308
:102230009887A987BA87C7010E94E6158B879C8774
:10224000CE0103966AE070E0AE014F5F5F4F22E07F
:1022500030E00E94800D9C0197FD02C029813A81E7
:10226000C9012C96CDBFDEBFCF91DF911F910F9199
:10227000FF90EF900895AF92BF92CF92DF92EF92CE
:10228000FF920F931F93DF93CF93CDB7DEB7659780
:10229000CDBFDEBF8091962E9091972E892B09F4A9
:1022A0008FC185E08983CE01019661E070E0AE01C7
:1022B0004C5F5F4F22E030E00E94800D97FD19C017
:1022C0008C819D81009799F4E091962EF091972E44
:1022D000278130852115310501F1868180FD1DC0E2
:1022E000816086838185928561E070E014C097FFEC
:1022F00014C0E091962EF091972E278130852115FC
:10230000310559F0868180FF08C08E7F86838185E4
:10231000928560E070E0F9011995A6E0AA2EB12C33
:10232000AC0EBD1EC50160E070E040E050E020E072
:1023300030E000E010E0FAE0EF2EF12CEC0EFD1E94
:10234000E2E0CE2ED12CCC0EDD1E0E94EC0D0097CB
:10235000A1F4E091962EF091972E238534852115D6
:10236000310521F1868181FD21C0826086838585CA
:102370009685B501F901199519C097FF15C0E0912F
:10238000962EF091972E238534852115310581F104
:10239000868181FF2DC08D7F86838585968560E04F
:1023A00070E0F901199524C0892B11F5E091962E62
:1023B000F091972E2785308921153105C9F08A8142
:1023C0009B81009731F481899289BE01665F7F4FBE
:1023D00007C08F5F9F4F61F48189928960E070E050
:1023E000F9011995E091962EF091972E1786108A93
:1023F000E091962EF091972E8681846086830091DD
:10240000982E1091992E23E1B22E9EE0C92ED12C48
:10241000CC0EDD1E82E1E82EF12CEC0EFD1E8CC0F0
:10242000D8018D919C91BE860E94E615888B998B70
:10243000C60164E070E0A70124E030E00E94800D56
:1024400097FD77C09D894A895B8957FD72C091309D
:10245000C9F4F801828180FD40C00780F085E02D3D
:102460003097D9F181608D7FD80112968C931297A5
:102470006D917C9111971B968D919C911C9741E0D9
:1024800050E056C09430B9F4F801828181FD25C036
:102490000780F085E02D309701F18E7F8260D801B2
:1024A00012968C9312976D917C9111971B968D913A
:1024B0009C911C973BC0933081F4D8011596ED9107
:1024C000FC911697309749F06D917C9111971B966E
:1024D0008D919C911C9719952CC04115510579F04F
:1024E000D8011996ED91FC911A97309741F06D91B2
:1024F0007C9111971D968D919C911E9719C09923DF
:10250000C1F4F801828180FF14C00184F285E02DBE
:10251000309779F08E7FD80112968C9312976D9137
:102520007C9111971D968D919C911E9740E050E0F3
:102530001995F801038114810115110509F070CF77
:10254000E091962EF091972E86818B7F8683A091C5
:10255000982EB091992EEE24FF2430C012968C91C3
:10256000129782FF23C0E114F10459F4E091982EF0
:10257000F091992E838194818093982E9093992E37
:1025800007C013968D919C911497F70183839483D0
:1025900013961C91139714960C911497CD010E94D9
:1025A000BC42212F302FC901DC0108C07D011396E8
:1025B0008C91139714969C919C01D901109771F6F8
:1025C0006596CDBFDEBFCF91DF911F910F91FF9038
:1025D000EF90DF90CF90BF90AF9008950F931F932F
:1025E000DF93CF9300D000D0CDB7DEB78C018FE062
:1025F0008B83C8010E94E6158D839E83CE010396CE
:1026000064E070E0AE014F5F5F4F22E030E00E9477
:10261000800D9C0197FD42C029813A8137FD3EC063
:102620006091982E7091992EDB0140E050E032C00D
:102630008D919C9111978017910721F5E091962E2D
:10264000F091972E868182FF07C012968C91129787
:10265000846012968C9320C04115510541F4FB0112
:10266000838194818093982E9093992E07C013961E
:102670008D919C911497FA0183839483CD010E94DC
:10268000BC420AC0AD0113968C91139714969C918D
:102690009C01D901109761F620E030E0C90126962F
:1026A000CDBFDEBFCF91DF911F910F910895EF92C3
:1026B000FF920F931F93DF93CF93CDB7DEB7C3582D
:1026C000D040CDBFDEBF9C018B017A010097C1F1E4
:1026D000FC0101900020E9F73197E81BF90BE03885
:1026E000F10570F5E091962EF091972E87859089EF
:1026F000892B19F022EF3FEF25C08AE08B83CE01B2
:102700000496B9010E949045CE01039661E870E0FD
:10271000AE014F5F5F4F22E030E00E94800D9C01D0
:1027200097FD10C029813A812115310559F4E091B6
:10273000962EF091972E0787108BE18AF28A02C0BD
:102740002EEF3FEFC901CD57DF4FCDBFDEBFCF9199
:10275000DF911F910F91FF90EF900895EF92FF92FC
:102760000F931F93DF93CF9300D000D0CDB7DEB788
:102770008C0181E090E06FE070E00E94F3417C0109
:10278000009719F40DEF1FEF42C084E18B83C8015D
:102790000E94E6158D839E83CE01039664E070E06F
:1027A000AE014F5F5F4F22E030E00E94800D8C0150
:1027B00097FF04C0C7010E94BC4229C089819A8149
:1027C00097FF06C0C7010E94BC4209811A811FC041
:1027D000F7018083918313821482828181608283D6
:1027E000E091982EF091992E309729F4E092982E4E
:1027F000F092992E09C0CF010380F481E02D30972B
:10280000D1F7FC01E382F482F70100811181C80154
:102810002696CDBFDEBFCF91DF911F910F91FF9024
:10282000EF900895EF92FF920F931F93DF93CF9352
:10283000CDB7DEB72597CDBFDEBF182F062F81E0BD
:1028400090E06FE070E00E94F3417C01009719F482
:102850000DEF1FEF3CC08BE08B831C830D83CE01FB
:10286000039663E070E0AE014F5F5F4F22E030E01F
:102870000E94800D8C0197FF04C0C7010E94BC42DA
:1028800026C089819A8197FF06C0C7010E94BC4279
:1028900009811A811CC0F7018083918313821482FD
:1028A000E091982EF091992E309729F4E092982E8D
:1028B000F092992E09C0CF010380F481E02D30976A
:1028C000D1F7FC01E382F482F70100811181C80194
:1028D0002596CDBFDEBFCF91DF911F910F91FF9065
:1028E000EF9008950F931F93DF93CF93CDB7DEB78B
:1028F000E397CDBFDEBF8C0186E08983CE010196D0
:1029000061E070E0AE014E5F5F4F22E330E00E9475
:10291000800D9C0197FD16C00115110589F0D801A5
:102920009196FE013C9686E001900D928150E1F770
:10293000D801FE01729681E201900D928150E1F77B
:102940002A813B81C901E396CDBFDEBFCF91DF91E4
:102950001F910F9108950F931F93DF93CF93CDB7DE
:10296000DEB7E397CDBFDEBF8C0186E08983CE0161
:10297000019661E070E0AE014E5F5F4F22E330E010
:102980000E94800D9C0197FD0DC00115110541F0BD
:10299000D801FE01369686E001900D928150E1F754
:1029A00020E030E0C901E396CDBFDEBFCF91DF91DB
:1029B0001F910F9108951F93DF93CF93CDB7DEB78B
:1029C000C856D040CDBFDEBF9C01142F86E6FE0165
:1029D0003396DF011D928A95E9F783E08B832115F9
:1029E000310541F0DE011796F90181E201900D9267
:1029F0008150E1F76115710531F0CE0188964FE302
:102A000050E00E94A545FE01E859FF4F1083CE011A
:102A1000039666E670E0AE014F5F5F4F22E030E064
:102A20000E94800D9C0197FD02C029813A81C90155
:102A3000C859DF4FCDBFDEBFCF91DF911F91089501
:102A4000CF92DF92EF92FF920F931F93DF93CF937A
:102A5000CDB7DEB76997CDBFDEBF8C017B016A01C0
:102A600082E08983CE01019661E070E0AE014E5FA5
:102A70005F4F28E130E00E94800D9C0197FD18C057
:102A80002A813B8137FD14C06E817F8188859985BD
:102A90000E941B16F8016083718382839383C701B0
:102AA000BE01665F7F4FA6010E94A5452A813B813A
:102AB000C9016996CDBFDEBFCF91DF911F910F9104
:102AC000FF90EF90DF90CF9008959F92AF92BF92CA
:102AD000CF92DF92EF92FF920F931F93DF93CF93EA
:102AE000CDB7DEB72B97CDBFDEBF5B016C01942E57
:102AF000D801C70147E749836CEB7EE26093962ECD
:102B00007093972E43E1FB0111924A95E9F72093C8
:102B1000BC2E3093BD2E0093BE2E1093BF2EE0929C
:102B2000C02EF092C12E8E010F5F1F4FB80141E001
:102B300050E0FD011995E091962EF091972E20819D
:102B4000318184819581B80141E050E0F901199506
:102B5000F02E012F0EC0E091962EF091972E20813D
:102B60003181848195816F2D702F41E050E0F90112
:102B7000199589818E3279F31C82C601B5010E94B4
:102B8000EE15688779878A879B879F82CE01049696
:102B900068E070E0AE014E5F5F4F22E030E00E94DF
:102BA000800D9C0197FD02C02A813B81C9012B96B3
:102BB000CDBFDEBFCF91DF911F910F91FF90EF90BE
:102BC000DF90CF90BF90AF909F900895282F892FCE
:102BD000922F0895282F892F922F0895EF92FF9218
:102BE0000F931F93E92EFF2400271127562F442708
:102BF00033272227E22AF32A042B152B2227362FEC
:102C0000472F582F207030705070E22AF32A042B7F
:102C1000152B672F782F892F9927607080709070FF
:102C2000E62AF72A082B192BB701C8011F910F912B
:102C3000FF90EF900895EF92FF920F931F93E92E6C
:102C4000FF2400271127562F442733272227E22A63
:102C5000F32A042B152B2227362F472F582F2070AD
:102C600030705070E22AF32A042B152B672F782F2F
:102C7000892F9927607080709070E62AF72A082BB8
:102C8000192BB701C8011F910F91FF90EF90089584
:102C90002F923F924F925F926F927F928F929F926C
:102CA000AF92BF92CF92DF92EF92FF920F931F935A
:102CB000DF93CF93CDB7DEB76497CDBFDEBFFC0106
:102CC000698B7A8B8081C82EDD24C7FCD0944E019D
:102CD0000894811C911C9E01235F3F4F2B8B3C8BE2
:102CE0008C2D80538A3008F067C130E3C316D104BD
:102CF00021F09AE0692E712C1BC031968081C82E7C
:102D0000DD24C7FCD09448E7C416D10441F058E54F
:102D1000C516D10421F088E0682E712C09C03196C7
:102D20008081C82EDD24C7FCD09400E1602E712C78
:102D30005F010894A11CB11CEE24FF24870113013C
:102D4000442437FC4094542CD50111979C2D8C2D94
:102D500080538A30A0F4C801B701A20191010E94FA
:102D60006441E0EDFFEFCE0EDF1E76010027F7FC99
:102D70000095102FE60EF71E081F191F2BC0F0E15B
:102D80006F16710489F52C2D2156263048F08C2DB4
:102D90008154863048F52A3118F021E430E002C031
:102DA00021E630E0D801C70114E0880F991FAA1F5F
:102DB000BB1F1A95D1F74AE050E0C40ED51EC21AC7
:102DC000D30A76010027F7FC0095102FE82AF92A8C
:102DD0000A2B1B2BF5018081C82EDD24C7FCD09463
:102DE0000894A11CB11CB0CFFEE2CF16D104C1F4EF
:102DF0002B893C898216930609F4DEC0F401E08237
:102E0000F1820283138324E030E0820E931EFD01E1
:102E1000319611968C91C82EDD24C7FCD09460CFDA
:102E2000C114D104F1F0903208F4C6C0C7FCC4C08C
:102E300030E2C316D104A9F04CE0C416D10489F0E5
:102E40005AE0C516D10469F08DE0C816D10449F0E6
:102E500099E0C916D10429F0EBE0CE16D10409F0AF
:102E6000ABC0CE0101969401281B390BC901959581
:102E700087959595879501968230910571F08330FD
:102E8000910524F4892B09F497C067C0833091051C
:102E9000B9F0049709F061C035C030E0E31630E0C6
:102EA000F30630E0030731E0130708F085C089819D
:102EB0009A81AB81BC81B82FAA279927882749C05E
:102EC00040E0E41640E0F40641E0040740E0140767
:102ED00008F072C02D813E814F815885A9013327AA
:102EE000222789819A81AB81BC81B82FAA27992793
:102EF0008827282B392B4A2B5B2BE22AF32A042B19
:102F0000152B2BC05FEFE516F1040105110511F03B
:102F100008F052C08D819E81AF81B885DC01992770
:102F2000882729813A814B815C81522F442733279E
:102F30002227822B932BA42BB52B29853A854B85F1
:102F40005C85542F432F322F2227822B932BA42BC7
:102F5000B52BE82AF92A0A2B1B2B89899A89892BF8
:102F600041F1212F332744275527BE2DAA27992722
:102F70008827282B392B4A2B5B2BB02FAF2D9E2D6A
:102F8000882780709070B070282B392B4A2B5B2BD0
:102F9000BB27A12F902F8F2D8070A070B070282B91
:102FA000392B4A2B5B2BE989FA89208331834283B1
:102FB000538321E030E002C020E030E0C901649694
:102FC000CDBFDEBFCF91DF911F910F91FF90EF90AA
:102FD000DF90CF90BF90AF909F908F907F906F9039
:102FE0005F904F903F902F900895AF92BF92CF92F5
:102FF000DF92EF92FF920F931F93DF93CF93CDB7A2
:10300000DEB72797CDBFDEBFFC0180819181A28111
:10301000B3818C839D83AE83BF8334E0E32EF12C98
:10302000EC0EFD1E0AE91EE26E010894C11CD11CC3
:103030005EE227E0A22EB12CAC0EBD1ED7014C9152
:1030400030E0842F6AE00E948341292F842F0E9460
:103050008341482FF601E30FF11D205D20833F5F80
:10306000882379F7932FF7011082D80106C03150D9
:10307000F601E30FF11D80818D933323C1F7F80131
:10308000E90FF11DDF015D938D01EA14FB0421F0CE
:103090000894E11CF11CD2CF10828AE99EE22796A7
:1030A000CDBFDEBFCF91DF911F910F91FF90EF90C9
:1030B000DF90CF90BF90AF900895CF93DF93EC0156
:1030C000DB0116964D935C931797EA81FB8130974D
:1030D00019F46A837B8309C0CF010084F185E02D58
:1030E0003097D1F7FC01A087B18718961D921C92EA
:1030F0001997DF91CF910895FB0146835783DC0137
:103100009E966D937C939F970895FC018081918199
:103110000895CF92DF92EF92FF920F931F93CF9378
:10312000DF938C016B017A01C0E0D0E012C0F601A0
:10313000EC0FFD1F6081772767FD7095D80116960B
:10314000ED91FC91179718968D919C91199719956F
:103150002196CE15DF055CF3DF91CF911F910F9182
:10316000FF90EF90DF90CF900895AF92BF92CF92F3
:10317000DF92EF92FF920F931F93CF93DF93FC01A7
:103180008B01DB018C91882319F4C0E0D0E02DC0C5
:10319000C281D381EE24FF24AA24BB2421C0C8808D
:1031A000D980C601B8010E9487450097F1F0D80187
:1031B0000D900020E9F71197A01BB10BC601B801D3
:1031C000AD010E949745009741F4EF2829F07E0158
:1031D00081E0A82EB12C01C07E010884D985C02DC4
:1031E0002097E9F6AB2809F4E701CE01DF91CF91F2
:1031F0001F910F91FF90EF90DF90CF90BF90AF9015
:103200000895CF93DF93EC01009749F08A859B8561
:10321000009711F00E94BC42CE010E94BC42DF9197
:10322000CF9108958F929F92AF92BF92CF92DF92EB
:10323000EF92FF920F931F93CF93DF934C01162FC2
:10324000072F81E090E061E070E00E94F341EC0123
:10325000009709F44AC0812F902F9C018901CC244A
:10326000DD2454010894A108B1083CC0EE24FF24D9
:10327000CA14DB041CF491E0E92EF12CDE010D9060
:103280000020E9F71197AC1BBD0BF80180819181FB
:10329000FC0101900020E9F73197E81BF90BAE0F14
:1032A000BF1F1196AE0DBF1DCE01BD010E9414437C
:1032B000009731F4CE010E94BC42C0E0D0E015C0BE
:1032C000EC01F801608171810E947C45EF2829F0B2
:1032D000CE0160E070E20E947C450894C11CD11CC4
:1032E0000E5F1F4FC814D9040CF2CE01DF91CF91AD
:1032F0001F910F91FF90EF90DF90CF90BF90AF9014
:103300009F908F900895CF92DF92EF92FF920F934C
:103310001F93DF93CF93CDB7DEB78E01005F1F4FB2
:1033200080EA90E00E940F42D82EC92E60EA70E039
:103330004E855F8598010E9438467C0197FF05C045
:103340002DEFE22E2FEFF22E1DC08D2D9C2D9C0116
:10335000890110C00F5F1F4F772767FD7095AC85FF
:10336000BD851696ED91FC91179718968D919C91BD
:1033700019971995F8016081662361F78D2D9C2DB1
:103380000E94BC42C701CF91DF911F910F91FF9026
:10339000EF90DF90CF900895EF92FF920F931F93DD
:1033A000CF93DF938C01DC011296CD91DC911397C2
:1033B00033E0E32E30E2F32E24C0288139818C8162
:1033C0009D81009711F482E090E2EDB7FEB7389747
:1033D000EDBFFEBF3196ADB7BEB711960D931C93EE
:1033E0001297E282F38224833583868397830E9437
:1033F00083190884D985C02DEDB7FEB73896EDBF87
:10340000FEBF2097D1F6DF91CF911F910F91FF90D2
:10341000EF9008958F929F92AF92BF92CF92DF92DA
:10342000EF92FF920F931F93CF93DF938C016B0169
:103430005A01922E832E6115710511F181E090E001
:1034400060E370E00E94F341EC017C010097E9F138
:103450000115110511F40EE010E20C831D8380EAC2
:1034600090E08C879D8781E090E060EA70E00E94A8
:10347000F3418A879B87009731F4CE010E94BC42BA
:10348000EE24FF2422C09A8A8B8ACE82DF82A8860D
:10349000B98690FC1AC000D000D0EDB7FEB73196C7
:1034A000ADB7BEB71196CD93DC93129780E190E251
:1034B000828393838C819D81848395830E94831969
:1034C0008DB79EB706968DBF9EBFC701DF91CF9186
:1034D0001F910F91FF90EF90DF90CF90BF90AF9032
:1034E0009F908F9008952F923F924F925F926F928C
:1034F0007F928F929F92AF92BF92CF92DF92EF9284
:10350000FF920F931F93DF93CF93CDB7DEB7C155D3
:10351000D040CDBFDEBF1C01142F052F62962FAF08
:103520006297832E2DB73EB7285030402DBF3EBF47
:10353000EDB7FEB73196ADB7BEB711968D939C939C
:10354000129784E190E28283938364837583629609
:10355000BFAD6297B68387820E948319212F302FD7
:10356000C9012C0166247724EDB7FEB7389693C0C5
:103570005301720100E010E081E090E08C0F9D1F8C
:10358000800F911FAC14BD0428F52DB73EB728500D
:1035900030402DBF3EBFEDB7FEB73196ADB7BEB7D9
:1035A00011968D939C93129780E590E0801B910B70
:1035B000828393832CE230E224833583D7018C917C
:1035C000868317820E94E345EDB7FEB73896EDBFBC
:1035D000FEBF04C062E370E20E9490450D5F1F4F82
:1035E0000894A11CB11C0894E11CF11C00331105C6
:1035F00019F6CE01C19666E370E20E949045520131
:103600008E010F5C1F4FEE24FF24C701860D971D0E
:103610008C159D05A0F4D5019C90892D992787FDD7
:1036200090950E943F4598012F5F3F4F892B19F0DD
:10363000F801908203C0EEE2D801EC93890108946E
:10364000E11CF11C0894A11CB11CF0E1EF16F1047F
:10365000E1F6D8011C9200D000D0EDB7FEB731964C
:10366000ADB7BEB711962D923C92129729E330E286
:103670002283338381E090E08C0F9D1F84839583A8
:103680000E948319A0E1B0E06A0E7B1E4A0E5B1E09
:10369000EDB7FEB73696EDBFFEBF6296CFAC629730
:1036A000D82C6C147D0408F463CFCF5ADF4FCDBF04
:1036B000DEBFCF91DF911F910F91FF90EF90DF90D0
:1036C000CF90BF90AF909F908F907F906F905F90C2
:1036D0004F903F902F9008951F93CF93DF93EC016D
:1036E000162F88899989892B31F18E859F858F398D
:1036F0009105F4F46E3659F0623719F06C3599F48F
:103700000DC0EA85FB85E80FF91F8DE005C0EA854D
:10371000FB85E80FF91F8AE0808305C0EA85FB85F9
:10372000E80FF91F60838E859F8501968E879F879E
:10373000188A198AFCC06A3099F16B3024F4683019
:1037400009F0C1C00DC06D3059F16C3509F0BBC036
:103750008A8982FF05C081E090E0888B998BE7C061
:103760008E859F85892B09F4E2C08A8981FD14C06A
:1037700000D00F92ADB7BEB71196CD93DC931297E0
:1037800081E490E213968D939C9314970E94831981
:103790000F900F900F900F908E859F850197C5C059
:1037A000EA85FB858E859F85E80FF91F10828A893F
:1037B00081FD10C000D00F92EDB7FEB7C183D28358
:1037C00085E490E2838394830E9483190F900F9085
:1037D0000F900F908A859B851C8A1D8A22E030E21B
:1037E0002E8B3F8B11C08C899D890B96FC01EE0FAF
:1037F000FF1FEC0FFD1F208331830A978C8B9D8B5D
:103800000C9749F080E090E060E070E20E9467452C
:103810009C01009741F76E897F89CE010E94B518FF
:10382000FC01009721F4EEA5FFA5309779F0868181
:103830009781888399836C897D89AE014A5E5F4F49
:103840000280F381E02DCE0119951DC0AE89BF899C
:103850008C918823C1F000D000D02DB73EB72F5FE8
:103860003F4FEDB7FEB7C183D28388E490E2F90100
:1038700082839383A483B5830E9483198DB79EB7F7
:1038800006968DBF9EBF1E861F868A8980FD4FC00B
:1038900000D000D0EDB7FEB73196ADB7BEB71196E8
:1038A000CD93DC93129780E190E2828393838C81A5
:1038B0009D81848395830E948319EDB7FEB7369668
:1038C000EDBFFEBF34C08E859F858F3991057CF595
:1038D000812F80528F3558F58A8981FD1CC000D018
:1038E00000D0EDB7FEB73196ADB7BEB71196CD9308
:1038F000DC9312978FE590E282839383812F99273F
:1039000087FD9095848395830E948319EDB7FEB758
:103910003696EDBFFEBFEA85FB858E859F85E80F55
:10392000F91F10838E859F8501968E879F87DF9173
:10393000CF911F910895CF92DF92EF92FF920F9354
:103940001F93DF93CF93CDB7DEB78E01045F1F4F78
:10395000F801E190F1908F0180EA90E00E940F421F
:10396000D82EC92E60EA70E0A70198010E9438465F
:103970007C0197FD05C08D2D9C2D9C0189010DC0FA
:103980008D2D9C2D0E94BC428DEFE82E8FEFF82EDE
:103990000CC00F5F1F4F0E94693FF8018081882390
:1039A000C1F78D2D9C2D0E94BC42C701CF91DF91A4
:1039B0001F910F91FF90EF90DF90CF9008952F927D
:1039C0003F924F925F926F927F928F929F92AF92AF
:1039D000BF92CF92DF92EF92FF920F931F93DF93EC
:1039E000CF93CDB7DEB7C155D040CDBFDEBF162FC8
:1039F000072F62964FAF6297852E00D000D0EDB7AB
:103A0000FEB731962EE730E2ADB7BEB711962D93D3
:103A10003C931297828393836296BFAD6297B4837F
:103A200055830E949B1C212F302FC9012C01662435
:103A30007724EDB7FEB73696EDBFFEBF91E3292E92
:103A4000312C2C0E3D1E8AC05301720100E010E0A3
:103A500081E090E08C0F9D1F800F911FAC14BD047E
:103A600028F52DB73EB7285030402DBF3EBFEDB7EB
:103A7000FEB73196ADB7BEB711968D939C93129752
:103A800080E590E0801B910B8283938326E930E2EE
:103A900024833583D7018C91868317820E94E34566
:103AA000EDB7FEB73896EDBFFEBF04C06CE970E21B
:103AB0000E9490450D5F1F4F0894A11CB11C0894F3
:103AC000E11CF11C0033110519F6C10160EA70E236
:103AD0000E94904552018101EE24FF24C701860D0A
:103AE000971D8C159D05A0F4D5019C90892D9927D3
:103AF00087FD90950E943F4598012F5F3F4F892B8E
:103B000019F0F801908203C0EEE2D801EC9389012C
:103B10000894E11CF11C0894A11CB11CF0E1EF1603
:103B2000F104E1F6D8011C9200D00F9223EA30E2B2
:103B3000EDB7FEB72183328381E090E08C0F9D1FAB
:103B4000838394830E949B1CA0E1B0E06A0E7B1EDD
:103B50004A0E5B1E0F900F900F900F906296CFACA5
:103B60006297D82C6C147D0408F46ECFCF5ADF4FC7
:103B7000CDBFDEBFCF91DF911F910F91FF90EF90EE
:103B8000DF90CF90BF90AF909F908F907F906F907D
:103B90005F904F903F902F90089597FD03C02BEAC0
:103BA00030E27EC0FC017696E631F10508F04AC0AD
:103BB000E650FF4FEE0FFF1F0590F491E02D199492
:103BC00023EB30E26DC026EC30E26AC026ED30E235
:103BD00067C02CEE30E264C02AEF30E261C028E01A
:103BE00031E25EC026E131E25BC025E231E258C03D
:103BF00027E331E255C025E431E252C02DE531E240
:103C00004FC02AE631E24CC023E731E249C02FE73A
:103C100031E246C024E831E243C02DE831E240C041
:103C20002CE931E23DC024EA31E23AC02CEA31E22B
:103C300037C02FEB31E234C02AEC31E231C022ED43
:103C400031E22EC00F920F9281EE91E2ADB7BEB776
:103C500011968D939C9312970E949B1C00D000D0CC
:103C6000EDB7FEB731968CEF91E2ADB7BEB71196C6
:103C70008D939C9312978EE092E28283938388E3E4
:103C800090E08483958383E29EE2868397830E94FB
:103C90009B1C25E332E2EDB7FEB73896EDBFFEBFC1
:103CA000C90108959C01E091AA2EF091AB2E82816A
:103CB0009381D90118968D939C931997848195814E
:103CC000FC016E9FC0016F9F900D7E9F900D11248F
:103CD00068EE73E00E948F41D9011A966D937C9330
:103CE0001B9716968D919C9117978E7F16968D93A4
:103CF0009C9317970895E091AA2EF091AB2E228104
:103D000033816481758188EE93E0AC01249FC0010A
:103D1000259F900D349F900D11240E948F41CB015F
:103D20000895E091AA2EF091AB2E309729F0828170
:103D300093810196828393830895CF93DF93C091FB
:103D4000AA2ED091AB2EEA81FB812C813D81AC0162
:103D5000429FC001439F900D529F900D112468EE29
:103D600073E00E948F416E0F7F1F8A819B818617AF
:103D70009707D8F3DF91CF9108959C018617970795
:103D800048F4CB01821B930B4817590718F421E024
:103D900030E012C06217730718F020E030E00CC06A
:103DA00080E090E020953095260F371F421753078B
:103DB00010F481E090E09C01C9010895681779072B
:103DC00030F49C0120953095260F371F03C09B01CE
:103DD000281B390BC9010895EF92FF920F931F938F
:103DE000CF93DF93E091AA2EF091AB2E868197813D
:103DF000816086839783C081D18108EE13E045C03E
:103E00006E817F8160FD3EC028853985E091AA2EB4
:103E1000F091AB2E42815381EA85FB85241735074B
:103E200030F4CA01821B930BE817F90750F04217D0
:103E3000530740F520953095240F351FE217F307FF
:103E400008F561606E837F836C817D81EA81FB81EF
:103E5000CE0119958E8181FF15C08A859B85E091E1
:103E6000AA2EF091AB2E648175819C01209FC00128
:103E7000219F900D309F900D11240E948F41CE0103
:103E80000E94521E0990D881C02D209709F0B8CF0A
:103E9000E091AA2EF091AB2E868197818E7F86834A
:103EA0009783C081D181EE24FF2423C08E8182FFBD
:103EB0001BC0E114F10449F4E091AA2EF091AB2E5D
:103EC000A081B1818D919C9103C088819981F70176
:103ED0008083918318810981CE010E94BC42212FE9
:103EE000302FC901EC0105C07E01888199819C01B8
:103EF000E9012097D9F6DF91CF911F910F91FF90A3
:103F0000EF900895CF93DF93EC010097E9F18E8154
:103F100082FF2CC00F920F928DE392E2ADB7BEB735
:103F200011968D939C9312970E949B1C00D000D0F9
:103F3000EDB7FEB7319688E592E2ADB7BEB7119600
:103F40008D939C93129784E892E2828393838AE60E
:103F500090E0848395838DE29EE2868397830E941E
:103F60009B1CEDB7FEB73896EDBFFEBFA091AA2E01
:103F7000B091AB2E16968C91169780FF08C08E815B
:103F80009F8184608E839F8320E030E023C04D9129
:103F90005C9111979A01E0E0F0E017C02C173D0703
:103FA00081F4309731F4FA01808191818D939C9353
:103FB00004C08881998180839183CE010E94BC4294
:103FC000E3CFF901808191819C012115310531F701
:103FD0002EEF3FEFC901DF91CF910895AF92BF92CD
:103FE000CF92DF92EF92FF920F931F93CF93DF93C5
:103FF0005C016B01EA0179014115510519F400E0FA
:1040000010E035C081E090E06CE070E00E94F34188
:10401000DC018C01009759F11296CD93DC93139734
:104020001496ED92FC921597CD2849F016968D9135
:104030009C911797826016968D939C931797C091C9
:10404000AA2ED091AB2EE881F981309719F4A8837C
:10405000B98309C0CF010190F081E02D3097D1F7ED
:10406000FC01A083B183CD01B5010E94521EC8019D
:10407000DF91CF911F910F91FF90EF90DF90CF9044
:10408000BF90AF900895CF93DF93EC01009719F4A0
:104090002EEF3FEF14C081E090E068E070E00E94F6
:1040A000F341FC018093AA2E9093AB2E009719F454
:1040B0002DEF3FEF04C0C483D58320E030E0C90179
:1040C000DF91CF910895CF92DF92EF92FF920F93FD
:1040D0001F93CF93DF93F801EC0188E0C03AD80733
:1040E000D9F4403885E2580780E0680780E0780717
:1040F00009F066C02830310509F062C081E0E81699
:10410000F10409F05DC00115110509F059C0CD2871
:1041100009F056C013E029C0CD2809F051C027305E
:104120003105A1F02830310520F42630310561F445
:1041300007C02830310531F02930310529F408C095
:1041400011E007C013E005C010E003C012E001C099
:1041500017E0E130F10531F0E130F10530F0329750
:1041600079F502C0106201C0106382E0E816F10424
:1041700009F418609A01AB0184E0220F331F441F39
:10418000551F8A95D1F7213088E4380788EE480713
:1041900081E0580720F02FEF3FEF8CE109C060E08D
:1041A00078E488EE91E00E94B6412150304088E1E9
:1041B0001C821D832E833F838C8320E030E002C06D
:1041C00026EF3FEFC901DF91CF911F910F91FF9033
:1041D000EF90DF90CF900895FC01818185FFFDCFA6
:1041E0006083E05AF84071F48091A10886FFFCCF0B
:1041F0008091A1088064E0EAF8E0818388EE93E092
:104200000197F1F70895EF92FF920F931F93CF93C9
:10421000DF937C0120E030E000EA18E0C8EED3E054
:1042200020C0FB01E20FF31FE081D70111968C91B2
:10423000119785FFFBCF8E2F992787FD90958C9343
:10424000A05AB84061F48091A10886FFFCCF80910C
:10425000A1088064F8018183CE010197F1F72F5FF7
:104260003F4F24173507ECF2CA01DF91CF911F9120
:104270000F91FF90EF900895FC01218130E02078AC
:104280003070C901089582309105A1F08330910505
:1042900028F4009761F00197B1F406C083309105CE
:1042A00061F0049781F40CC02DEA32E23AC02FEAA3
:1042B00032E237C021EB32E234C023EB32E231C0CC
:1042C00025EB32E22EC00F920F9287EB92E2ADB750
:1042D000BEB711968D939C9312970E949B1C00D0A1
:1042E00000D0EDB7FEB7319682ED92E2ADB7BEB722
:1042F00011968D939C93129784EE92E2828393831E
:1043000089EB90E0848395838BE39EE28683978399
:104310000E949B1C22E133E2EDB7FEB73896EDBF59
:10432000FEBFC9010895EF92FF920F931F93182FBC
:10433000092F7B010E947B1EE12FF02FEF2819F03F
:1043400006EF1FEF06C0818187FFFDCF8081082F18
:1043500010E0C8011F910F91FF90EF900895CF9248
:10436000DF92EF92FF920F931F93CF93DF936C0135
:104370007B018A01C0E0D0E00AC0C60160E070E0C5
:104380000E949321F701EC0FFD1F80832196C01737
:10439000D1079CF3C801DF91CF911F910F91FF903E
:1043A000EF90DF90CF90089580E090E008959C0119
:1043B000883091054CF481E090E002C0880F991F8D
:1043C0002A95E2F780938706089587E0E0EAF0E017
:1043D00082830E94E8070E94200883E090E060E169
:1043E0000E94D30784E090E060E10E94D3077894B4
:1043F00080E090E008952091B02E3091B12E2151AF
:104400003140C9010895FF920F931F938C01F62E3E
:1044100060E070E0CB01BA0126E631E040E050E018
:104420000E9464412091AE2E3091AF2E40E050E0CA
:104430000E94B6412093B02E3093B12E3FB7F8942E
:10444000F801208181E090E002C0880F991FFA9462
:10445000E2F7880F880F822B80833FBF1F910F9157
:10446000FF9008950F931F93DF93CF93CDB7DEB7DF
:104470002A97CDBFDEBFFE01349687E0DF011D9293
:104480008A95E9F78E010F5F1F4F83E0D8011D92D7
:104490008A95E9F72D819E819F7C86E08887217E21
:1044A0002D831F8291609E8380E092E0BF010E9475
:1044B000F80C80E092E063E072E20E94C70B198280
:1044C0001A828B81807F81608B8380E092E060E044
:1044D000A8010E945C0C82E06FE20E949022182FDB
:1044E00000E082E06EE20E94902290E0082B192BFF
:1044F0000093AE2E1093AF2E80E092E00E94FC0B52
:104500009FB7F894E0E0F2E08081846080839FBFF1
:104510002A96CDBFDEBFCF91DF911F910F910895F5
:104520004091CA01E62FFF278093CA0184914093EE
:10453000CA0108952DB73EB7245130402DBF3EBF6C
:10454000EDB7FEB73196ADB7BEB711968D939C937C
:10455000129783E193E28283938381E090E0A0E06D
:10456000B0E084839583A683B78380879187A287F1
:10457000B38783E090E0A0E0B0E084879587A687CA
:10458000B78783E091E0A1E0B0E0808B918BA28BB4
:10459000B38B0E9483192DB73EB72C5E3F4F2DBFC2
:1045A0003EBF08952DB73EB7285030402DBF3EBFC7
:1045B000EDB7FEB73196ADB7BEB711968D939C930C
:1045C000129780E393E282839383648375834683A7
:1045D00057830E9483192DB73EB7285F3F4F2DBFE9
:1045E0003EBF0895CF92DF92EF92FF920F931F93F9
:1045F000DF93CF93CDB7DEB76497CDBFDEBF6C013D
:10460000CE010196BE016B5F7F4F40E150E00E94FA
:1046100020158C0197FF05C021E5E22E23E2F22E42
:1046200004C095E5E92E93E2F92EC8010E94CD1D44
:104630002DB73EB72A5030402DBF3EBFEDB7FEB775
:104640003196ADB7BEB71196CD92DC92129728E5A0
:1046500033E222833383E482F582068317838087E3
:1046600091870E94831929813A814B815C818DB7A2
:104670009EB70C978DBF9EBFEDB7FEB73196ADB715
:10468000BEB71196CD92DC92129784E693E28283B4
:104690009383CA01AA27BB2784839583A683B78304
:1046A000832F90E0A0E0B0E080879187A287B38756
:1046B000DA01C9019070A070B07084879587A687D1
:1046C000B787208B318B428B538BCE010596848B21
:1046D000958B0E9483192DB73EB72A5E3F4F2DBFA1
:1046E0003EBF6496CDBFDEBFCF91DF911F910F918A
:1046F000FF90EF90DF90CF900895EF92FF920F938D
:104700001F93CF93DF938C01FA0162307105BCF1E6
:10471000828193816AED73E2A8010E945713EC0134
:1047200097FF05C041E5E42E43E2F42E04C035E5D1
:10473000E32E33E2F32ECE010E94CD1D2DB73EB7FE
:104740002A5030402DBF3EBFEDB7FEB73196ADB712
:10475000BEB711960D931C9312972AE833E2228379
:104760003383E482F582C683D783808791870E9452
:104770008319EDB7FEB73A96EDBFFEBF14C000D067
:104780000F92ADB7BEB711968D939C93129787E9A0
:1047900093E213968D939C9314970E9483190F9024
:1047A0000F900F900F90DF91CF911F910F91FF907D
:1047B000EF9008950F931F93182F092F611571051E
:1047C000A9F400D00F92EDB7FEB73196ADB7BEB7E2
:1047D00011968C93918389EB93E2828393830E9459
:1047E00083190F900F900F900F901AC0CB010E9469
:1047F000F51700D000D0EDB7FEB73196ADB7BEB714
:1048000011961C93018325ED33E222833383848345
:1048100095830E9483198DB79EB706968DBF9EBF64
:104820001F910F910895CF92DF92EF92FF920F9315
:104830001F93DF93CF9300D000D0CDB7DEB76C01CC
:10484000FA01623071050CF457C002811381C8016E
:10485000BE016F5F7F4F40E050E00E94F0439B013C
:10486000AC0189819A818017910709F05AC044C030
:1048700065E5E62E63E2F62EC8010E94CD1D2DB738
:104880003EB72A5030402DBF3EBFEDB7FEB7319640
:10489000ADB7BEB71196CD92DC92129728E533E200
:1048A00022833383E482F58206831783808791878E
:1048B0000E948319EDB7FEB73A96EDBFFEBFCE0159
:1048C00003960E94F51700D000D0EDB7FEB73196E1
:1048D000ADB7BEB71196CD92DC92129727EE33E2B8
:1048E00022833383848395830E948319EDB7FEB7B7
:1048F0003696EDBFFEBF23C000D00F92ADB7BEB756
:104900001196CD92DC92129781EF93E213968D93DC
:104910009C9314970E9483190F900F900F900F9003
:104920000EC0C901BE016D5F7F4F0E94500F8C0108
:1049300097FF9ECF51E5E52E53E2F52E9DCF2696AB
:10494000CDBFDEBFCF91DF911F910F91FF90EF9010
:10495000DF90CF9008952F923F924F925F926F9287
:104960007F928F929F92AF92BF92CF92DF92EF92FF
:10497000FF920F931F93DF93CF93CDB7DEB72A97A4
:10498000CDBFDEBF3C016B017A01643071050CF4D0
:10499000DAC0DA0112960D911C911397C8015E01DD
:1049A0000894A11CB11CB50140E050E00E94F04306
:1049B0006F83788789819A818017910709F0D8C021
:1049C000C2C0F70106811781C801B50140E050E07F
:1049D0000E94F0439B01AC0189819A818017910765
:1049E00009F4B1C0122F032F37FDADC028E030E02D
:1049F000E20EF31EC6010497B7010E9412194C0182
:104A0000009709F476C019870A87DC010D90002011
:104A1000E9F77D010894E108F108E81AF90AC201F2
:104A20000E94F517EDB7FEB73A97EDBFFEBF31967E
:104A3000ADB7BEB711966D927C92129720E134E229
:104A400022833383E482F5828683978310870187EC
:104A50000E948319AA24BB24EDB7FEB73A96EDBF96
:104A6000FEBF1201ACE24A2EA4E25A2E35C0670105
:104A7000CA18DB08B4016A0D7B1D8F819885A601D9
:104A8000910109851A850E94840F8C0197FF04C04B
:104A9000C4010E94BC422FC02DB73EB72850304001
:104AA0002DBF3EBFEDB7FEB73196ADB7BEB711967D
:104AB0006D927C9212974282538284839583C81AA6
:104AC000D90AC682D7820E948319A00EB11EEDB703
:104AD000FEB73896EDBFFEBFAE14BF0444F2C4016A
:104AE0000E94BC42F5E5EF2EF3E2FF2E00E010E05D
:104AF00006C00DEF1FEFE1E5EE2EE3E2FE2EC8014A
:104B00000E94CD1D2DB73EB72A5030402DBF3EBF6D
:104B1000EDB7FEB73196ADB7BEB711966D927C92E8
:104B200012972AE833E222833383E482F5820683F4
:104B30001783808791870E948319EDB7FEB73A9655
:104B4000EDBFFEBF23C000D00F92ADB7BEB7119628
:104B50006D927C92129781E494E213968D939C93CC
:104B600014970E9483190F900F900F900F900EC012
:104B700073E0472E512C4C0E5D1EF7018481958108
:104B8000B2010E944816892BF1F21BCF2A96CDBFA5
:104B9000DEBFCF91DF911F910F91FF90EF90DF90DB
:104BA000CF90BF90AF909F908F907F906F905F90CD
:104BB0004F903F902F9008952F923F924F925F9287
:104BC0006F927F928F929F92AF92BF92CF92DF921D
:104BD000EF92FF920F931F93DF93CF930F920F9259
:104BE000CDB7DEB73C016B017A01633071050CF47F
:104BF000A6C0DA0112960D911C911397C801BE014F
:104C00006F5F7F4F40E050E00E94F0431B018981BD
:104C10009A818017910709F0A7C091C0D4010D9027
:104C20000020E9F77D010894E108F108E818F90887
:104C300000D000D0EDB7FEB73196ADB7BEB7119634
:104C40006D927C92129781E794E282839383E4824F
:104C5000F5820E948319AA24BB24EDB7FEB73696CD
:104C6000EDBFFEBF0CE2402E04E2502E31C06701C2
:104C7000CA18DB08B4016A0D7B1DC101A6010E94A0
:104C8000E20F8C0197FF04C0C4010E94BC422FC0F8
:104C90002DB73EB7285030402DBF3EBFEDB7FEB711
:104CA0003196ADB7BEB711966D927C921297428243
:104CB000538284839583C81AD90AC682D7820E94F8
:104CC0008319A00EB11EEDB7FEB73896EDBFFEBF3B
:104CD000AE14BF0464F2C4010E94BC4215E5E12E8B
:104CE00013E2F12E00E010E006C00DEF1FEFB1E57A
:104CF000EB2EB3E2FB2EC8010E94CD1D2DB73EB7AF
:104D00002A5030402DBF3EBFEDB7FEB73196ADB74C
:104D1000BEB711966D927C9212972AE833E22283F5
:104D20003383E482F58206831783808791870E940C
:104D30008319EDB7FEB73A96EDBFFEBF23C000D092
:104D40000F92ADB7BEB711966D927C92129784E820
:104D500094E213968D939C9314970E9483190F905D
:104D60000F900F900F900EC0E4E0F0E0EE0EFF1EEB
:104D7000C6010297B7010E9412194C01009709F071
:104D80004DCFB3CF0F900F90CF91DF911F910F9127
:104D9000FF90EF90DF90CF90BF90AF909F908F905B
:104DA0007F906F905F904F903F902F900895CF929B
:104DB000DF92EF92FF920F931F93DF93CF930F92A7
:104DC0000F92CDB7DEB76C01FA0162307105D4F1F4
:104DD00002811381C801BE016F5F7F4F40E050E048
:104DE0000E94F0439B01AC0189819A818017910751
:104DF000F1F528C095E5E92E93E2F92EC8010E944D
:104E0000CD1D2DB73EB72A5030402DBF3EBFEDB768
:104E1000FEB73196ADB7BEB71196CD92DC92129720
:104E20002AE833E222833383E482F5820683178300
:104E3000808791870E948319EDB7FEB73A96EDBF40
:104E4000FEBF20C000D00F92ADB7BEB71196CD9275
:104E5000DC92129786EA94E213968D939C931497B2
:104E60000E9483190F900F900F900F900BC0C901F3
:104E70000E94EE128C0197FFBDCF81E5E82E83E200
:104E8000F82EBCCF0F900F90CF91DF911F910F9113
:104E9000FF90EF90DF90CF9008954F925F926F92C6
:104EA0007F928F929F92AF92BF92CF92DF92EF92BA
:104EB000FF920F931F93DF93CF9300D000D0CDB715
:104EC000DEB72C017A01643071050CF45FC0DA01A1
:104ED00012960D911C911397C8014E010894811CE4
:104EE000911CB40140E050E00E94F0435B016C0172
:104EF00089819A818017910709F05DC047C0F70149
:104F000006811781C801B40140E050E00E94F043DF
:104F10009B01AC0189819A8180179107B9F137FD16
:104F200035C0C501B301A9010E9470108C0197FF23
:104F300005C041E5E42E43E2F42E04C035E5E32E3E
:104F400033E2F32EC8010E94CD1D2DB73EB72A5083
:104F500030402DBF3EBFEDB7FEB73196ADB7BEB7FF
:104F600011964D925C9212972AE833E222833383A2
:104F7000E482F58206831783808791870E948319D4
:104F8000EDB7FEB73A96EDBFFEBF23C000D00F923B
:104F9000ADB7BEB711964D925C9212978EEB94E22C
:104FA00013968D939C9314970E9483190F900F90E2
:104FB0000F900F900EC023E0622E712C6C0E7D1EA0
:104FC000F70184819581B3010E944816892BF1F283
:104FD00096CF2696CDBFDEBFCF91DF911F910F9167
:104FE000FF90EF90DF90CF90BF90AF909F908F9009
:104FF0007F906F905F904F9008954F925F926F9265
:105000007F928F929F92AF92BF92CF92DF92EF9258
:10501000FF920F931F93DF93CF930F920F92CDB711
:10502000DEB73C015B014A01623071050CF45FC0E0
:10503000DA0112960D911C911397C8012E01089464
:10504000411C511CB20140E050E00E94F0436B0152
:105050007C0189819A818017910709F05DC047C062
:10506000F40104811581C801B20140E050E00E94C2
:10507000F0439B01AC0189819A8180179107B9F1B6
:10508000B901C60147EA58E293010E94C0108C01A1
:1050900097FF05C061E5E62E63E2F62E04C055E5F4
:1050A000E52E53E2F52EC8010E94CD1D2DB73EB767
:1050B0002A5030402DBF3EBFEDB7FEB73196ADB799
:1050C000BEB711966D927C9212972AE833E2228342
:1050D0003383E482F58206831783808791870E9459
:1050E0008319EDB7FEB73A96EDBFFEBF1DC000D0E5
:1050F0000F92ADB7BEB711966D927C92129784EE67
:1051000094E213968D939C9314970E9483190F90A9
:105110000F900F900F9008C0B2E0AB16B10409F0E9
:105120009FCF61E070E0ADCF0F900F90CF91DF91F6
:105130001F910F91FF90EF90DF90CF90BF90AF90B5
:105140009F908F907F906F905F904F900895EF9217
:10515000FF920F931F93CF93DF93F82EE92E8B01CD
:1051600000D000D0EDB7FEB73196ADB7BEB71196FF
:105170008C93918387E095E2828393836483758324
:105180000E9483192DB73EB72A5F3F4F2DBF3EBF08
:10519000C8010E94AE13EC011816190674F462EDF2
:1051A00072E24F2D5E2D0E944A0DCE016BE079E236
:1051B0004F2D5E2D0E94650D05C0009719F001E589
:1051C00013E202C005E513E2CE010E94CD1DADB78A
:1051D000BEB71A97ADBFBEBFEDB7FEB731961196F9
:1051E000FC92E1822AE833E222833383048315832D
:1051F000C683D783808791870E9483192DB73EB7D6
:10520000265F3F4F2DBF3EBFDF91CF911F910F9182
:10521000FF90EF900895AF92BF92CF92DF92EF92FE
:10522000FF920F931F93DF93CF93CDB7DEB7C05498
:10523000D040CDBFDEBF5C017B018A014115510525
:1052400019F42BE235E202C02DE335E28DB79EB7AB
:105250000A978DBF9EBFEDB7FEB73196ADB7BEB70B
:105260001196AC92B1828EE395E282839383E482BD
:10527000F58206831783208731870E9483198DB7B3
:105280009EB70A968DBF9EBF6E010894C11CD11CAB
:1052900017C00134110510F4A80102C040E450E029
:1052A000C701B6010E9429109C01181619068CF737
:1052B000081B190BC5016CE575E2A6010E94731A63
:1052C0001016110634F3C05CDF4FCDBFDEBFCF91A7
:1052D000DF911F910F91FF90EF90DF90CF90BF90E3
:1052E000AF9008954F925F926F927F928F929F92AC
:1052F000AF92BF92CF92DF92EF92FF920F931F93E4
:10530000DF93CF9300D000D0CDB7DEB72C017A0168
:10531000643071050CF45FC0DA0112960D911C9196
:105320001397C8014E010894811C911CB40140E000
:1053300050E00E94F0435B016C0189819A818017E3
:10534000910709F05DC047C0F70106811781C801C8
:10535000B40140E050E00E94F0439B01AC01898120
:105360009A8180179107B9F137FD35C0C501B301A6
:10537000A9010E94FF108C0197FF05C0F1E5EF2EF7
:10538000F3E2FF2E04C0E5E5EE2EE3E2FE2EC801B7
:105390000E94CD1D2DB73EB72A5030402DBF3EBFD5
:1053A000EDB7FEB73196ADB7BEB711964D925C9290
:1053B00012972AE833E222833383E482F58206835C
:1053C0001783808791870E948319EDB7FEB73A96BD
:1053D000EDBFFEBF23C000D00F92ADB7BEB7119690
:1053E0004D925C9212978FE595E213968D939C9364
:1053F00014970E9483190F900F900F900F900EC07A
:1054000073E0672E712C6C0E7D1EF70184819581EF
:10541000B3010E944816892BF1F296CF2696CDBF94
:10542000DEBFCF91DF911F910F91FF90EF90DF9042
:10543000CF90BF90AF909F908F907F906F905F9034
:105440004F9008958F929F92AF92BF92CF92DF922A
:10545000EF92FF920F931F93DF93CF930F920F92D0
:10546000CDB7DEB76C015B014A01623071050CF407
:105470007EC0DA0112960D911C911397C80162E863
:1054800075E20E948745009719F4EE24FF2416C0A8
:10549000C80169E875E20E948745009721F401E0A0
:1054A000E02EF12C0BC0C8016FE875E20E94874521
:1054B000009709F05CC012E0E12EF12CB2E0AB16CF
:1054C000B10419F460E070E014C0F40104811581A6
:1054D000C801BE016F5F7F4F40E050E00E94F04383
:1054E0009B01AC0189819A818017910709F43FC023
:1054F000B901C7010E9412148C0162ED72E2A6018B
:105500000E944A0DC8016BE079E2A6010E94650D78
:1055100017FF05C0B1E5EB2EB3E2FB2E04C0A5E5F5
:10552000EA2EA3E2FA2EC8010E94CD1D2DB73EB788
:105530002A5030402DBF3EBFEDB7FEB73196ADB714
:10554000BEB71196CD92DC9212972AE833E22283FD
:105550003383E482F58206831783808791870E94D4
:105560008319EDB7FEB73A96EDBFFEBF14C000D069
:105570000F92ADB7BEB71196CD92DC92129783E928
:1055800095E213968D939C9314970E9483190F9024
:105590000F900F900F900F900F90CF91DF911F9170
:1055A0000F91FF90EF90DF90CF90BF90AF909F90C2
:1055B0008F9008950F931F93DF93CF930F920F92C5
:1055C000CDB7DEB78C01CE0101960E94820EAC01F0
:1055D00097FF03C021E533E202C025E533E28DB732
:1055E0009EB70A978DBF9EBFEDB7FEB73196ADB798
:1055F000BEB711960D931C93129781EC95E28283AE
:105600009383248335834683578389819A81808756
:1056100091870E9483198DB79EB70A968DBF9EBF52
:105620000F900F90CF91DF911F910F910895CF921E
:10563000DF92EF92FF920F931F93DF93CF930F921E
:105640000F92CDB7DEB76C01FA0162307105D4F16B
:1056500002811381C801BE016F5F7F4F40E050E0BF
:105660000E94F0439B01AC0189819A8180179107C8
:10567000F1F528C095E5E92E93E2F92EC8010E94C4
:10568000CD1D2DB73EB72A5030402DBF3EBFEDB7E0
:10569000FEB73196ADB7BEB71196CD92DC92129798
:1056A0002AE833E222833383E482F5820683178378
:1056B000808791870E948319EDB7FEB73A96EDBFB8
:1056C000FEBF20C000D00F92ADB7BEB71196CD92ED
:1056D000DC92129786ED95E213968D939C93149726
:1056E0000E9483190F900F900F900F900BC0C9016B
:1056F0000E94190F8C0197FFBDCF81E5E82E83E250
:10570000F82EBCCF0F900F90CF91DF911F910F918A
:10571000FF90EF90DF90CF9008950F931F93DF934A
:10572000CF93CDB7DEB76097CDBFDEBF8C01CE0182
:105730000196BE016B5F7F4FAE01475F5F4F9E01D9
:10574000235F3F4F0E949E0EAC0197FF03C021E5EF
:1057500033E202C025E533E28DB79EB708978DBFCF
:105760009EBFEDB7FEB73196ADB7BEB711960D939C
:105770001C9312978EEE95E2828393832483358364
:10578000468357830E9483198DB79EB708968DBFB5
:105790009EBFCE0101960E94F51700D000D0EDB754
:1057A000FEB73196ADB7BEB711960D931C93129705
:1057B00026EF35E222833383848395830E94831905
:1057C0008DB79EB706968DBF9EBFCE0105960E94EF
:1057D000F51700D000D0EDB7FEB73196ADB7BEB724
:1057E00011960D931C9312972DEF35E2228333838C
:1057F000848395830E9483198DB79EB706968DBFCB
:105800009EBFCE0109960E94F51700D000D0EDB7DB
:10581000FEB73196ADB7BEB711960D931C93129794
:1058200026E036E222833383848395830E948319A2
:105830008DB79EB706968DBF9EBFCE010D960E9476
:10584000F51700D000D0EDB7FEB73196ADB7BEB7B3
:1058500011960D931C9312972DE036E22283338329
:10586000848395830E9483198DB79EB706968DBF5A
:105870009EBF6096CDBFDEBFCF91DF911F910F918C
:105880000895CF92DF92EF92FF920F931F93DF93D1
:10589000CF93CDB7DEB76097CDBFDEBF6C018B0174
:1058A0007A0180911B2E90911C2EA0911D2EB091FB
:1058B0001E2E8D839E83AF83B88789879A87AB8797
:1058C000BC878D879E87AF87B88B623071050CF4DB
:1058D00075C0DA0112968D919C911397BE016F5F8E
:1058E0007F4F0E944816892B09F468C002301105C9
:1058F00041F1F70184819581BE016B5F7F4F0E946A
:105900004816892B09F45AC003301105D1F0D7018C
:1059100016968D919C911797BE01675F7F4F0E94ED
:105920004816892B09F44AC00530110554F0F701D7
:1059300080859185BE01635F7F4F0E944816892B49
:10594000E9F1CE010196BE016B5F7F4FAE01475F6B
:105950005F4F9E01235F3F4F0E94290F8C0197FFED
:1059600005C031E5E32E33E2F32E04C025E5E22E37
:1059700023E2F22EC8010E94CD1D2DB73EB72A505A
:1059800030402DBF3EBFEDB7FEB73196ADB7BEB7C5
:105990001196CD92DC9212972AE833E22283338368
:1059A000E482F58206831783808791870E9483199A
:1059B000EDB7FEB73A96EDBFFEBF14C000D00F9210
:1059C000ADB7BEB71196CD92DC92129787E196E201
:1059D00013968D939C9314970E9483190F900F90A8
:1059E0000F900F906096CDBFDEBFCF91DF911F91DA
:1059F0000F91FF90EF90DF90CF9008958F929F923C
:105A0000AF92BF92CF92DF92EF92FF920F931F93CC
:105A1000DF93CF93CDB7DEB7C854D040CDBFDEBF44
:105A20005C018E010E5D1F4FC8010E9472146C0153
:105A300052E4E52EF12CEC0EFD1ED7014C91CE0167
:105A40000196B80150E00E946C45F701E080D7FE56
:105A500003C001E513E202C005E513E2EE2029F0E0
:105A60004E010894811C911C04C042E4842E46E23D
:105A7000942EFE01ED5BFF4F2081FE01EC5BFF4F9A
:105A80003081FE01EB5BFF4F4081FE01EA5BFF4F7F
:105A90005081FE01E95BFF4F6081FE01E85BFF4F33
:105AA0007081FE01EE0DF11D11828DB79EB74697F4
:105AB0008DBF9EBFEDB7FEB73196ADB7BEB711969D
:105AC000AD92BC92129786E496E28283938304831C
:105AD0001583C682D7828086918622871386348773
:105AE000158646871786508B118A628B138A748BB2
:105AF000158A0E948319EDB7FEB77696EDBFFEBFFB
:105B0000C85BDF4FCDBFDEBFCF91DF911F910F91FB
:105B1000FF90EF90DF90CF90BF90AF909F908F90CD
:105B20000895AC01DC010D900020E9F71197A81B46
:105B3000B90BFB01A0A3CB01BA014A2F50E00E9490
:105B40006C4581E090E008950F931F93DF93CF930E
:105B500000D000D0CDB7DEB78C01CE0101960E94F7
:105B6000AB14AC0197FF03C021E533E202C025E589
:105B700033E28DB79EB744978DBF9EBFEDB7FEB79A
:105B80003196ADB7BEB711960D931C93129781E76E
:105B900096E2828393832483358346835783898166
:105BA000808711868A81828713868B8184871586F8
:105BB0008C81868717868D81808B118A8E81828B5E
:105BC000138A0E9483198DB79EB744968DBF9EBFDE
:105BD0002696CDBFDEBFCF91DF911F910F91089523
:105BE000EF92FF920F931F93CF93DF937C010E945C
:105BF000320FEC0197FF03C001E513E202C005E597
:105C000013E2CE010E94CD1D2DB73EB72A50304081
:105C10002DBF3EBFEDB7FEB73196ADB7BEB71196FB
:105C2000ED92FC9212972AE833E2228333830483B5
:105C30001583C683D783808791870E9483192DB7E8
:105C40003EB7265F3F4F2DBF3EBFDF91CF911F91E3
:105C50000F91FF90EF900895AF92BF92CF92DF9295
:105C6000EF92FF920F931F93DF93CF93CDB7DEB7E1
:105C7000A397CDBFDEBF5C017A01E3E0CE2ED12C2D
:105C8000CC0EDD1E81E2D6011D928A95E9F76430C3
:105C90007105FCF0FA0182819381B6010E94912D79
:105CA000892B09F471C0D70116960D911C91179795
:105CB000C801BE016F5F7F4F40E050E00E94F0439B
:105CC0009B01AC0189819A818017910709F071C00D
:105CD0005BC06330710581F4FA0182819381B60162
:105CE0000E94912D892B09F44FC0D70114966D9114
:105CF0007C911597C60114C06230710551F4FA0108
:105D000082819381B6010E94912D892BE9F1C60110
:105D100005C061307105C1F580E090E060E070E0A1
:105D200040E050E00E94DB148C0197FF05C071E554
:105D3000E72E73E2F72E04C065E5E62E63E2F62E49
:105D4000C8010E94CD1D2DB73EB72A5030402DBF4F
:105D50003EBFEDB7FEB73196ADB7BEB71196AD9267
:105D6000BC9212972AE833E222833383E482F582DD
:105D700006831783808791870E948319EDB7FEB74A
:105D80003A96EDBFFEBF1BC000D00F92ADB7BEB7B5
:105D90001196AD92BC92129789E996E213968D9373
:105DA0009C9314970E9483190F900F900F900F905F
:105DB00006C0F70164817581C601A901B3CFA3961E
:105DC000CDBFDEBFCF91DF911F910F91FF90EF907C
:105DD000DF90CF90BF90AF9008954F925F926F92F7
:105DE0007F928F929F92AF92BF92CF92DF92EF926B
:105DF000FF920F931F93CF93DF93582E492EEB0101
:105E00003A014801590100D00F92EDB7FEB7319623
:105E1000ADB7BEB711968C9391838DE299E28283E0
:105E200093830E9483190F900F900F900F902097EB
:105E3000E1F0CE010E94CD1DEDB7FEB73897EDBF62
:105E4000FEBF3196ADB7BEB711965C92418220E39A
:105E500039E222833383C483D583868397830E9468
:105E60008319EDB7FEB738965BC081149104A10485
:105E7000B10409F440C06301EE24D7FCE094FE2C89
:105E80002DB73EB7225130402DBF3EBF0DB71EB7D4
:105E90000F5F1F4FADB7BEB711965C92F8014182FC
:105EA00083E499E28283938364827582D801169693
:105EB0008D929D92AD92BC921997C701B601A50132
:105EC00094010E94B641F8012287338744875587A1
:105ED000C701B601A50194010E94B641D8011E96E2
:105EE0006D937D938D939C9351970E948319EDB789
:105EF000FEB7729615C000D000D0EDB7FEB7319650
:105F0000ADB7BEB711965C92418286E799E2828373
:105F10009383648275820E948319EDB7FEB736962B
:105F2000EDBFFEBFDF91CF911F910F91FF90EF90DA
:105F3000DF90CF90BF90AF909F908F907F906F90A9
:105F40005F904F9008950F931F93CF93DF93182F77
:105F5000092FEB0100D00F92EDB7FEB73196ADB728
:105F6000BEB711968C9391838CE999E282839383D7
:105F70000E9483190F900F900F900F901C161D0612
:105F8000DCF4CE0160E570E00E94A341892BA1F40E
:105F900000D00F92EDB7FEB73196ADB7BEB71196F0
:105FA0001C9301838DE299E2828393830E9483197B
:105FB0000F900F900F900F90DF91CF911F910F9145
:105FC0000895AF92BF92CF92DF92EF92FF920F931C
:105FD0001F93CF93DF93EC01B62EA72E8889998962
:105FE000892B71F08C819D812E813F81AC01429F74
:105FF000C001439F900D529F900D11246C0104C06D
:10600000CA88DB88EC88FD886C857D8588859985C4
:106010000E94DE1EEA8DFB8D309749F08C0120E056
:1060200030E08C8D9D8D6B2D7A2DA60119958A817E
:106030009B810E94BC42888199810E94EE128889CE
:106040009989892B21F48E899F890E94EE12CE01B5
:106050000E94BC428B2D9A2DDF91CF911F910F9101
:10606000FF90EF90DF90CF90BF90AF9008958F9208
:106070009F92AF92BF92CF92DF92EF92FF920F93D7
:106080001F93CF93DF934C017B016A01590181E09B
:1060900090E06EE170E00E94F341EC01009719F48A
:1060A00080E090E010C0EC82FD82C88ED98EAA8E6E
:1060B000BB8E0C8F1D8FC7010E940F428A839B836A
:1060C000009731F4CE016DEF7FEF0E94E12F23C0E6
:1060D00080E090E060E070E00E941214BC018883D0
:1060E000998397FD14C06BE17EE2A4010E94FF102A
:1060F000BC0197FD0CC08881998161E070E048E99E
:1061000050E39E010E94C010BC0197FF02C0CE0167
:10611000DCCF88819981DF91CF911F910F91FF9002
:10612000EF90DF90CF90BF90AF909F908F900895A9
:10613000CF93DF93EC01CB010E94AE13BC018E8B99
:106140009F8B97FF04C0CE010E94E12F14C065E031
:1061500071E3AE010E944A0D8E899F896EEB70E358
:10616000AE010E94650D0E947B1EA0E0B0E0888712
:106170009987AA87BB87DF91CF910895CF93DF934B
:106180009B01EC0188899989892BE1F5452B61F404
:106190000E947B1EA0E0B0E08C879D87AE87BF8702
:1061A000CE0160E070E00BC06A817B814C815D8133
:1061B000C9010E942910BC0197FF04C0CE010E94B2
:1061C000E12F20C0EE81FF813196EE83FF839C0199
:1061D000442737FD4095542F8A899B89AC89BD8916
:1061E000820F931FA41FB51F8A8B9B8BAC8BBD8B1B
:1061F000288D398D2115310529F08C8D9D8DBF019C
:10620000F9011995DF91CF9108954F925F926F92A6
:106210007F928F929F92AF92BF92CF92DF92EF9236
:10622000FF920F931F93CF93DF93EC01452B19F44B
:106230006CEF7FEFA6C088899989892B61F50F9251
:106240000F928EE999E2ADB7BEB711968D939C93EC
:1062500012970E949B1C00D000D0EDB7FEB731967C
:1062600089EB99E2ADB7BEB711968D939C931297C7
:1062700084ED99E28283938382EB90E0848395831B
:106280008AE49EE2868397830E949B1CEDB7FEB74B
:106290003896EDBFFEBF0E947B1EA0E0B0E088876D
:1062A0009987AA87BB87EE24FF244EE9442E49E252
:1062B000542E35EE632E39E2732E24ED822E29E220
:1062C000922E95E1A92E91E0B92E82E5C82E8EE29C
:1062D000D82E44C06A817B81600F711F401B510B17
:1062E000888199810E94E20FBC0197FD2EC0080FA2
:1062F000191F4C815D810417150760F304171507FA
:1063000009F452C00F920F92ADB7BEB711964D92DD
:106310005C9212970E949B1C00D000D0EDB7FEB794
:106320003196ADB7BEB711966D927C92129782826C
:106330009382A482B582C682D7820E949B1CEDB74D
:10634000FEB73896EDBFFEBF2FC0CE011AC08C8DB0
:106350009D8DB70119950894E11CF11C8E819F81D8
:10636000E816F90618F400E010E0C3CF0E947B1E87
:10637000A0E0B0E08C879D87AE87BF87CE0160E04C
:1063800070E00E94E12FDF91CF911F910F91FF905C
:10639000EF90DF90CF90BF90AF909F908F907F90C5
:1063A0006F905F904F900895E88DF98D309779F652
:1063B000D2CF4F925F926F927F928F929F92AF92C5
:1063C000BF92CF92DF92EF92FF920F931F93CF93E2
:1063D000DF932C013B014A0159014115510509F494
:1063E00055C02115310509F451C06115710509F435
:1063F0004DC081E090E06EE170E00E94F341EC015D
:10640000009719F44DEF5FEF43C08E829F82AC82FC
:10641000BD82088F198FEA8EFB8ECC8EDD8E81E0D7
:1064200090E0888B998BC5010E940F428A839B83E1
:10643000009721F4CE016DEF7FEF13C080E090E074
:1064400060E070E00E941214BC018883998397FD7C
:1064500007C0B201A3010E947010BC0197FF05C0E4
:10646000CE010E94E12FAC0113C08881998165E0C3
:1064700071E3AE010E944A0D888199816EEB70E351
:10648000AE010E94650D4881598102C04EEF5FEF59
:10649000CA01DF91CF911F910F91FF90EF90DF9094
:1064A000CF90BF90AF909F908F907F906F905F90B4
:1064B0004F9008952F923F924F925F926F927F92EA
:1064C0008F929F92AF92BF92CF92DF92EF92FF9204
:1064D0000F931F93DF93CF9300D000D0CDB7DEB7DB
:1064E0005C013B016A0180911B2E90911C2EA091B2
:1064F0001D2EB0911E2E89839A83AB83BC8301E04D
:1065000010E038E8832E33E1932E20E034E02D8331
:106510003E83412C24E0522E2224332470C0F80103
:10652000EE0FFF1FEC0DFD1DE080F180C70169E05B
:106530007AE20E948745009789F40F5F1F4F061586
:1065400017050CF0EEC0F801EE0FFF1FEC0DFD1D5E
:10655000808191810E941F454C014FC0C7016CE0B2
:106560007AE20E948745009791F40F5F1F4F06154E
:1065700017050CF0D6C0F801EE0FFF1FEC0DFD1D46
:10658000808191810E941F458D839E8336C0C70103
:106590006FE07AE20E948745009789F40F5F1F4FF2
:1065A000061517050CF0BDC0F801EE0FFF1FEC0D2E
:1065B000FD1D808191810E941F452C011EC0C701D5
:1065C00062E17AE20E948745009721F4F1E02F2EE4
:1065D000312C13C0C70165E17AE20E94874500971C
:1065E00019F42224332409C0C701BE016F5F7F4F15
:1065F0000E944816892B09F494C00F5F1F4F06159F
:1066000017050CF48CCF21143104C9F089819A81CB
:10661000AB81BC810097A105B10509F482C0CE0110
:106620000196B4014D815E81920103EA1FE2EDEE15
:10663000EE2EEEE2FE2E65010E94D93109C0C401A2
:10664000B20143EA5FE22DEE3EE285010E9437305F
:106650008C0197FF1BC00E94CD1DADB7BEB71A9726
:10666000ADBFBEBFEDB7FEB731961196AD92BC92ED
:10667000129728E13AE22283338325E23AE2248327
:106680003583068317838087918743C0232859F178
:10669000CE0101960E94F5172DB73EB72E5030401F
:1066A0002DBF3EBFEDB7FEB73196ADB7BEB7119661
:1066B000AD92BC92129729E23AE22283338384831B
:1066C0009583868297822D813E81208731874286FD
:1066D0005386048715870E9483198DB79EB70E963F
:1066E0008DBF9EBF32C0ADB7BEB71A97ADBFBEBF9C
:1066F000EDB7FEB731961196AD92BC9212978AE52E
:106700009AE28283938384829582468257820087AD
:1067100011870E948319EDB7FEB73A96EDBFFEBF11
:1067200014C000D00F92ADB7BEB71196AD92BC9217
:10673000129785E89AE213968D939C9314970E9482
:1067400083190F900F900F900F902696CDBFDEBF4C
:10675000CF91DF911F910F91FF90EF90DF90CF903D
:10676000BF90AF909F908F907F906F905F904F9071
:106770003F902F9008952F923F924F925F926F9289
:106780007F928F929F92AF92BF92CF92DF92EF92C1
:10679000FF920F931F93DF93CF93CDB7DEB7EE97A2
:1067A000CDBFDEBF9C016DAF7EAFDE011196EAE585
:1067B000FEE284E301900D928150E1F7D901ED9062
:1067C000FD900D911C91C801B70120E831E541E031
:1067D00050E00E94B641C901DA015C016D01C801B7
:1067E000B70120E831E541E050E00E94B641AC013C
:1067F000CB01DA017C018D010DC080E891E5A1E0BB
:10680000B0E0E80EF91E0A1F1B1F0894A108B1088A
:10681000C108D10817FDF1CF0DC080E89EEAAEEFA8
:10682000BFEFE80EF91E0A1F1B1F0894A11CB11C24
:10683000C11CD11C90E8E91691E5F90691E0090721
:1068400090E0190750F7C801B70120E13EE040E0B1
:1068500050E00E94D841ADADBEAD12962C93C80158
:10686000B70120E13EE040E050E00E94D841162F01
:10687000072FF82EE92E2CE330E040E050E00E9494
:10688000D841EDADFEAD2183612F702F8F2D9E2D50
:106890002CE330E040E050E00E94D841ADADBEAD09
:1068A0006C93C601B5016C5F7F4F8F4F9F4F27E000
:1068B00030E040E050E00E94D841EDADFEAD618790
:1068C000E2EB2E2EE7E03E2E412C512C2EC1C601CC
:1068D000B5012DE631E040E050E00E94D841390199
:1068E0004A01EE24FF248701C601B5012DE631E0FF
:1068F00040E050E00E94D84197FF05C071E0E72ECC
:10690000F12C012D112DD401C3018E199F09A00B6B
:10691000B10B820D931DA41DB51D8DAB9EABAFAB0E
:10692000B8AF4201310108946108710881089108EB
:106930000197A109B10989AF9AAFABAFBCAFC40150
:10694000B30124E030E040E050E00E94D8417901FA
:106950008A01C401B3012CE93FEF4FEF5FEF0E94C2
:10696000D841E20EF31E041F151FEA0CFB1C0C1D80
:106970001D1DC401B30120E931E040E050E00E9458
:10698000D841E20EF31E041F151FAA24BB24650183
:10699000C401B30124E630E040E050E00E94D84159
:1069A00097FF05C061E0A62EB12CC12CD12CAE0CF6
:1069B000BF1CC01ED11EEE24FF248701C401B301F9
:1069C00024E030E040E050E00E94D84197FF05C04D
:1069D00051E0E52EF12C012D112DAE18BF08C00A93
:1069E000D10AEE24FF248701C401B30120E931E07C
:1069F00040E050E00E94D84197FF05C041E0E42EFE
:106A0000F12C012D112DD601C5018E199F09A00B66
:106A1000B10B7C018D0169AD7AAD8BAD9CAD20E7EA
:106A20003EEF4FEF5FEF0E94D841E20EF31E041FCE
:106A3000151F69AD7AAD8BAD9CAD24E630E040E02A
:106A400050E00E94D841E20EF31E041F151F69ADED
:106A50007AAD8BAD9CAD24E030E040E050E00E9488
:106A6000D841E21AF30A040B150B8DA99EA9AFA910
:106A7000B8AD281A390A4A0A5B0AC201B1012DE6EB
:106A800031E040E050E00E946441E60EF71E081F2E
:106A9000191FAA24BB24650169AD7AAD8BAD9CADED
:106AA00020E931E040E050E00E94D84197FF05C066
:106AB00031E0A32EB12CC12CD12CAE0CBF1CC01EBA
:106AC000D11EEE24FF24870169AD7AAD8BAD9CAD5C
:106AD00024E030E040E050E00E94D84197FF05C03C
:106AE00021E0E22EF12C012D112DAE0CBF1CC01E99
:106AF000D11EEE24FF24870169AD7AAD8BAD9CAD2C
:106B000024E630E040E050E00E94D84197FF05C005
:106B100091E0E92EF12C012D112DAE18BF08C00A0D
:106B2000D10A2DA83EA84FA858ACD7FCD0CE83E000
:106B3000E82EF12C012D112DE220F3200421152146
:106B4000E114F10401051105F9F4C201B10124E6D3
:106B500030E040E050E00E94D841611571058105A8
:106B6000910569F4C201B10120E931E040E050E053
:106B70000E94D841611571058105910529F48EE6C1
:106B800091E0A0E0B0E004C08DE691E0A0E0B0E0CC
:106B9000A816B906CA06DB060CF099CEC1018C56C0
:106BA0009740ADADBEAD15968D939C9316971796F5
:106BB000AD92BC921897E114F1040105110519F08A
:106BC00020E030E022C0C201B10124E630E040E024
:106BD00050E00E94D841611571058105910519F0B9
:106BE00021E030E012C000E010E0C201B10120E974
:106BF00031E040E050E00E94D84161157105810507
:106C0000910511F401E010E098018AE190E0FC01A7
:106C10002E9FC0012F9F900D3E9F900D1124FE01CD
:106C20003196E80FF91F2BE030E040E050E004C05F
:106C30002150304040405040868997893297A0E0EB
:106C4000B0E0A816B906CA06DB0694F3EDADFEADBA
:106C50002483A81AB90ACA0ADB0A8A2D8F5F8383A4
:106C600081E090E0EE96CDBFDEBFCF91DF911F9126
:106C70000F91FF90EF90DF90CF90BF90AF909F90DB
:106C80008F907F906F905F904F903F902F900895DE
:106C90000F931F93CF93DF93182F092FDB01EA0186
:106CA0006115710509F5CA010E94CD1D2DB73EB7CA
:106CB000285030402DBF3EBFEDB7FEB73196ADB77F
:106CC000BEB711961C93018326EB3AE222833383ED
:106CD00084839583C683D7830E948319CDB7DEB79B
:106CE0002896CDBFDEBF3AC02DB73EB72051304009
:106CF0002DBF3EBFEDB7FEB73196CDB7DEB7898366
:106D0000918386ED9AE28283938315968D919C916F
:106D100016978459984F8483958314968C91149771
:106D200090E001968683978313968C9113978087C2
:106D3000118612968C9112978287138611968C91E8
:106D40001197848715868C91868717860E948319F0
:106D50002DB73EB7205F3F4F2DBF3EBFDF91CF9194
:106D60001F910F910895CF93DF93EC018C819D814A
:106D70001816190614F40E94EE128E819F81009756
:106D800011F00E94821FCE010E94BC42DF91CF9180
:106D900008956F927F928F929F92AF92BF92CF92FF
:106DA000DF92EF92FF920F931F93DF93CF93CDB7B4
:106DB000DEB7E097CDBFDEBF4C018B015A013E012B
:106DC0000894611C711C80E3F30111928A95E9F724
:106DD00083E2898381E090E068E070E00E94F34103
:106DE0007C01009719F40DEF1FEF3FC081E090E0A8
:106DF00060E070E00E9412146C011816190684F508
:106E0000F70100831183A282B3828483958388E88B
:106E100093E160E070E04AEB57E397010E94EE1FB8
:106E2000F70186839783892BD9F0C601B4014BE71C
:106E300050E00E9470108C010097A1F4C6016EEC26
:106E400077E3A7010E94650D97FD08C0C601B30155
:106E500040E350E00E94E20F97FF07C08C0102C0A0
:106E60000DEF1FEFC7010E94B336C801E096CDBFFA
:106E7000DEBFCF91DF911F910F91FF90EF90DF90D8
:106E8000CF90BF90AF909F908F907F906F9008951C
:106E9000CF92DF92EF92FF920F931F93DF93CF93E6
:106EA00000D00F92CDB7DEB77C01FA0162307105D8
:106EB0000CF440C0828193818E010F5F1F4FB80197
:106EC0000E944816892BB1F1C80168E476E3A70156
:106ED0000E94C9368C0197FF05C0A0E0CA2EABE224
:106EE000DA2E04C0F4E0CF2EFBE2DF2EC8010E94B0
:106EF000CD1D2DB73EB72A5030402DBF3EBFEDB758
:106F0000FEB73196ADB7BEB71196ED92FC921297CF
:106F100027E03BE222833383C482D5820683178332
:106F2000808791870E948319EDB7FEB73A96EDBF2F
:106F3000FEBF14C000D00F92ADB7BEB71196ED9250
:106F4000FC92129784E19BE213968D939C93149785
:106F50000E9483190F900F900F900F902496CDBF31
:106F6000DEBFCF91DF911F910F91FF90EF90DF90E7
:106F7000CF900895CF93DF93EB01E881F9813097AB
:106F800039F08A819B8160E070E04FEE5FEF1995E8
:106F9000CE010E94B336DF91CF910895AF92BF9298
:106FA000CF92DF92EF92FF920F931F93DF93CF93D5
:106FB000CDB7DEB72E97CDBFDEBF6B017A018C0156
:106FC0004033510538F4AA24BB2480EFC82E8FEF3C
:106FD000D82E2EC0CA010E940F425C01009729F4EE
:106FE000BDEFCB2EBFEFDB2E23C0C601B501A7013D
:106FF0000E9429106C018E159F05D1F4D501909641
:107000006D917D918D919C9193970E941B16605874
:107010007E478A4A934869837A838B839C83F8945A
:10702000CE010196BE016B5F7F4F0E94BB33789407
:10703000D801ED91FC911197309749F012968D91FE
:107040009C911397BE016B5F7F4FA6011995C501F7
:107050000E94BC42C8010E94B3362E96CDBFDEBF4F
:10706000CF91DF911F910F91FF90EF90DF90CF9024
:10707000BF90AF900895CF92DF92EF92FF920F935F
:107080001F93D82EC92ECB018A0179010E94F517D2
:1070900000D000D0EDB7FEB73196ADB7BEB71196B0
:1070A000DC92C1822BE43BE2228333838483958389
:1070B0000E9483190F920F92EDB7FEB73196ADB7CC
:1070C000BEB71196DC92C18288E69BE282839383ED
:1070D00004831583E682F7820E9483198DB79EB7D9
:1070E00008968DBF9EBF1F910F91FF90EF90DF908C
:1070F000CF900895CF92DF92EF92FF920F931F935C
:10710000CF93DF93D82EC92EEB017901011511051C
:10711000A1F4CA010E94F5172DB73EB72A5030409E
:107120002DBF3EBFEDB7FEB73196ADB7BEB71196D6
:10713000DC92C1822EE83BE213C003301105F9F462
:10714000CA010E94F517ADB7BEB71A97ADBFBEBF53
:10715000EDB7FEB731961196DC92C1822EEA3BE282
:1071600022833383C483D58386839783E086F18625
:107170000E9483192DB73EB7265F3F4F20C0CA013A
:107180000E94F517ADB7BEB71C97ADBFBEBFEDB738
:10719000FEB731961196DC92C1822BEE3BE2228340
:1071A0003383C483D58386839783E086F186028701
:1071B00013870E9483192DB73EB7245F3F4F2DBF21
:1071C0003EBFDF91CF911F910F91FF90EF90DF9025
:1071D000CF900895CF93DF93EC01888D998D181689
:1071E000190614F40E94EE128A8D9B8D009711F0FF
:1071F0000E94821F8C819D810E94BC42CE010E9410
:10720000BC42DF91CF9108954F925F926F927F922F
:107210008F929F92AF92BF92CF92DF92EF92FF92A6
:107220000F931F93CF93DF935C014B01D42EC52E98
:107230003901280181E090E06CE170E00E94F341A7
:10724000EC01009709F445C00D2D1C2DB801685FB5
:107250007F4F81E090E00E94F3418C839D830097F3
:10726000A9F182E090E061E070E00E941214888F42
:10727000998F1816190654F567E07BE3AE010E945A
:10728000650DF50180819181A281B3818883998305
:10729000AA83BB838A8A9B8A0E831F831E861F86CE
:1072A000688679864A865B86EC86FD8680E090E07B
:1072B00060E070E040E65AE39E010E94EE1F8A8F74
:1072C0009B8F892B19F020E030E005C0CE010E9491
:1072D000EA382DEF3FEFC901DF91CF911F910F9158
:1072E000FF90EF90DF90CF90BF90AF909F908F90E6
:1072F0007F906F905F904F9008952F923F924F92A2
:107300005F926F927F928F929F92AF92BF92CF9235
:10731000DF92EF92FF920F931F93DF93CF9300D0F2
:107320000F92CDB7DEB74C015B016A0180911B2E35
:1073300090911C2EA0911D2EB0911E2E89839A83B0
:10734000AB83BC8301E010E063E0462E512C50E299
:10735000652E712C1E010894211C311C40C0F801BF
:10736000EE0FFF1FEC0DFD1DE080F180C70163E112
:107370007CE20E948745009789F40F5F1F4F0A1532
:107380001B050CF073C0F801EE0FFF1FEC0DFD1D87
:10739000808191810E941F452C011FC0C70166E1B9
:1073A0007CE20E948745009789F40F5F1F4F0A1502
:1073B0001B050CF05BC0F801EE0FFF1FEC0DFD1D6F
:1073C000808191810E941F453C0107C0C701B10126
:1073D0000E944816892B09F449C00F5F1F4F0A15F8
:1073E0001B050CF4BCCF89819A81AB81BC810097CD
:1073F000A105B105D9F1CE010196B201A3012AE799
:1074000038E30BE318E374010E9404398C0197FF01
:1074100005C099E1E92E9CE2F92E04C08DE1E82E29
:107420008CE2F82EC8010E94CD1D2DB73EB72A5020
:1074300030402DBF3EBFEDB7FEB73196ADB7BEB7FA
:1074400011968D929C92129720E23CE22283338324
:10745000E482F58206831783808791870E948319CF
:10746000EDB7FEB73A96EDBFFEBF14C000D00F9245
:10747000ADB7BEB711968D929C9212978DE29CE2A9
:1074800013968D939C9314970E9483190F900F90DD
:107490000F900F902496CDBFDEBFCF91DF911F914B
:1074A0000F91FF90EF90DF90CF90BF90AF909F90A3
:1074B0008F907F906F905F904F903F902F900895A6
:1074C000CF92DF92EF92FF920F931F93CF93DF93B0
:1074D000EB010C811D81288939898A899B892817AC
:1074E000390779F4EA85FB85309739F04C895D8955
:1074F0002E893F898C859D851995CE010E94EA3899
:107500007DC0CE80DF8088E090E0C80ED91E88E084
:10751000F80180831182128213828E859F850E94DA
:10752000E615F80184839583888999890E94E61578
:10753000F80186839783760120E030E040E050E058
:1075400011C0708160E0818190E0862B972B32968C
:10755000A0E0B0E0280F391F4A1F5B1F8EEF9FEF9E
:10756000E80EF91E92E0E916F10458F7C6018E7F85
:10757000F801E80FF91FC816D90641F0908180E0A4
:10758000A0E0B0E0280F391F4A1F5B1FCA01AA27DD
:10759000BB2740705070280F391F4A1F5B1F40FFE8
:1075A00009C0CA01AA27BB2740705070280F391F95
:1075B0004A1F5B1FC9010E94E61580959095F8014E
:1075C00082839383888D998DB801A6019E0100E086
:1075D00010E00E94840F8C159D0529F48C899D89EB
:1075E00001968C8B9D8B8A8D9B8D68EE73E00E943B
:1075F000521E888999890196888B998BDF91CF914A
:107600001F910F91FF90EF90DF90CF9008958F9290
:107610009F92AF92BF92CF92DF92EF92FF920F9321
:107620001F93CF93DF93E82E992E8B01EA01CA01B5
:107630000E940F426C010097C1F1C801B601AE0172
:107640000E9429105C018C179D0779F58CE1A81622
:10765000B10458F1CE2DD92D86010C5E1F4FF801D3
:10766000848195810E94EA152E853F8582179307B4
:10767000E1F48E899F8901968E8B9F8B88849984F3
:107680008114910491F0EC84FD84F8018681978146
:107690000E94EA159C01A601445F5F4FF80100813A
:1076A000C701B50110E0F4011995C6010E94BC4262
:1076B000DF91CF911F910F91FF90EF90DF90CF90CE
:1076C000BF90AF909F908F9008952F923F924F92CE
:1076D0005F926F927F928F929F92AF92BF92CF9262
:1076E000DF92EF92FF920F931F93DF93CF9300D01F
:1076F0000F92CDB7DEB75C013B0129833A832801A5
:107700006115710519F48B839C830BC0FB010190FB
:10771000F081E02DE80FF91FEB83FC83FB01108261
:1077200011828A018824992415010894211C311C96
:1077300050C0EB81FC819081992309F452C0F8017B
:107740008081C92EDD24C7FCD0944114510431F04E
:10775000E82EFF24E7FCF094C60109C0992787FDB5
:1077600090950E944D457C01C6010E944D45E8164A
:10777000F90629F1F8018081F501F08041145104E6
:1077800049F0C82EDD24C7FCD0948F2D992787FDA2
:1077900090950CC0992787FD90950E944D456C01EE
:1077A0008F2D992787FD90950E944D45C816D906C3
:1077B00019F0AB82BC8208C02B823C8205C08B8151
:1077C0009C8101968B839C830F5F1F4F0894811CC3
:1077D000911CE981FA818E169F0608F4AACF00E079
:1077E00010E06114710439F08B819C818A199B0926
:1077F000F30180839183C8012496CDBFDEBFCF9172
:10780000DF911F910F91FF90EF90DF90CF90BF908D
:10781000AF909F908F907F906F905F904F903F9030
:107820002F900895CF92DF92EF92FF920F931F93C4
:10783000CF93DF936C017B01DB010D900020E9F712
:107840008D0101501040061B170BC0E0D0E00EC0A8
:10785000B7016C0F7D1FA8014C1B5D0BC6010E9478
:10786000E20F9C0197FD07C0C80FD91FC017D107B1
:107870007CF320E030E0C901DF91CF911F910F919F
:10788000FF90EF90DF90CF9008958F929F92AF92EC
:10789000BF92CF92DF92EF92FF920F931F93CF93FD
:1078A000DF934C015B016A0180E091E00E940F428E
:1078B000F82EE92E00E010E021C0E601C01BD10B3C
:1078C00081E0C130D80714F0C0E0D1E0B501600F0D
:1078D000711F8F2D9E2DAE010E945545C4016F2D45
:1078E0007E2DAE010E94E20FEC0197FF05C08F2DA7
:1078F0009E2D0E94BC420BC0080F191F0C151D05C0
:10790000E4F28F2D9E2D0E94BC42C0E0D0E0CE015B
:10791000DF91CF911F910F91FF90EF90DF90CF906B
:10792000BF90AF909F908F900895EF92FF920F932A
:107930001F937C018B01CB010E945E45AC01C70106
:10794000B8010E94453C1F910F91FF90EF90089560
:10795000EF92FF920F931F93DF93CF93CDB7DEB7D4
:10796000AC97CDBFDEBF7C01009719F42FEF3FEF3E
:10797000E2C08EE49FE2A1E4B0E08B8F9C8FAD8FDC
:10798000BE8FFE017F968EE0DF011D928A95E9F79A
:10799000C70167E876E00E94953C9C0197FDCBC04B
:1079A0008E010F5F1F4FC80160E070E040E050E0C3
:1079B00020E030E00E949E0E892B19F00EE51CE2BB
:1079C00004C0C8010E94F5178C01C70162E776E088
:1079D0000E94953C9C0197FDAEC0C701B8010E9472
:1079E000123C9C0197FDA7C0C70167E576E00E94A5
:1079F000953C9C0197FD9FC0CE0105960E94AB145B
:107A0000892B99F52DB73EB7225130402DBF3EBF8F
:107A1000EDB7FEB73196CE014B96ADB7BEB7119616
:107A20008D939C93129782E190E08283938382E608
:107A30009CE2848395838D81868317828E818087E3
:107A400011868F818287138688858487158689852C
:107A5000868717868A85808B118A0E94E3452DB719
:107A60003EB72E5E3F4F2DBF3EBFC70161E476E0BB
:107A70000E94953C9C0197FD5EC0C701BE01655EFA
:107A80007F4F0E94123C9C0197FD55C0C70166E2E2
:107A900076E00E94953C9C0197FD4DC0C70160E1D6
:107AA00076E00E94953C9C0197FD45C00E94FB2119
:107AB000ADB7BEB71897ADBFBEBFEDB7FEB7319635
:107AC0008E01055F1F4F11960D931C93129720E1B5
:107AD00030E02283338320E83CE2248335838683AD
:107AE00097830E94E3452DB73EB7285F3F4F2DBFD8
:107AF0003EBFC701B8010E94123C9C0197FD1BC00C
:107B0000C70165EF75E00E94953C9C0197FD13C08D
:107B1000C70168EC73E00E94953C9C0197FD0BC087
:107B2000C70160E272E00E94953C9C01181619069C
:107B300014F420E030E0C901AC96CDBFDEBFCF9198
:107B4000DF911F910F91FF90EF900895EF92FF92B8
:107B50000F931F93DF93CF930F920F92CDB7DEB7A2
:107B60008C017B0165E87CE20E948745009799F1D2
:107B7000C80167E87CE20E948745009761F1C8016F
:107B80006AE87CE24CE050E00E949745009741F59E
:107B900000D000D0EDB7FEB73196045F1F4FADB7F0
:107BA000BEB711960D931C93129787E99CE28283CE
:107BB0009383CE010196848395830E941B462DB743
:107BC0003EB72A5F3F4F2DBF3EBF892B21F08981F1
:107BD0009A810E94D721C7010E94A83C9C012FC016
:107BE000C80164EA7CE20E9487450097A1F3C801BE
:107BF00060EB7CE20E948745009781F4C7016FEC3F
:107C00007DE00E94953C9C0197FD19C0C7016AEE7A
:107C100078E045EE54E00E94453C0BC0E114F104CD
:107C200019F42FEF3FEF0BC0C7016BE07EE00E941D
:107C3000953C9C011816190614F420E030E0C901A7
:107C40000F900F90CF91DF911F910F91FF90EF90C8
:107C50000895CF93DF93EC018E819F81009731F0DF
:107C60000E94BC421E821F82188619868A819B81CF
:107C7000009721F00E94EE121A821B82DF91CF91B1
:107C80000895CF93DF93EC010E94293E888199816A
:107C9000009711F00E94EE12CE010E94BC42DF91CB
:107CA000CF910895EF92FF920F931F93CF93DF939D
:107CB0007C0181E090E06AE070E00E94F341EC0119
:107CC0008C01009739F180E090E060E070E00E9464
:107CD00012148883998397FD12C06BE17EE2A7019D
:107CE0000E94FF10892B59F48881998161E070E02E
:107CF00042E95EE39E010E94C010892B59F0888101
:107D00009981009711F00E94EE12CE010E94BC42B0
:107D100000E010E0C801DF91CF911F910F91FF901B
:107D2000EF9008950F931F93CF93DF93EC018A8117
:107D30009B81892B19F0CE010E94293E888199816F
:107D40000E94AE138C0197FD0DC062E57FE3AE018A
:107D50000E944A0DC80167EB7EE3AE010E94650DEB
:107D60000A831B83DF91CF911F910F910895CF92CA
:107D7000DF92EF92FF920F931F93CF93DF938B01CC
:107D8000EA017C014115510519F40E94293E81C088
:107D9000CA010E940F42D82EC92EC8016D2D7C2D1C
:107DA000AE010E94291097FD6BC0F701C085D185F7
:107DB000C80FD91FF2E0C130DF0710F0C0E0D2E0F9
:107DC000F70186819781BE010E9414439C01F7014F
:107DD0008683978380859185280F391FFE01E81BD4
:107DE000F90BC9016D2D7C2DAF010E946C45F70187
:107DF000C087D187468157818AEB9CE260E070E0C2
:107E00009E0101E010E00E94653BFC01009779F1C2
:107E10001082F701C681D781CE016DEB7CE244E090
:107E200050E00E949745009741F5249601C02196A5
:107E30008881992787FD90950E944545892BB9F740
:107E40001C2F0D2F01C021968881992787FD9095C1
:107E50000E944545892BB9F31882F701628173812D
:107E6000812F902F0E94A63D892B39F40EC0F70177
:107E7000808591858050924019F4C7010E94293E67
:107E80008D2D9C2D0E94BC4204C0C7010E94293E3A
:107E9000EECFDF91CF911F910F91FF90EF90DF9088
:107EA000CF900895DF93CF9300D00F92CDB7DEB778
:107EB000452B39F0CB01BE016F5F7F4F0E94500F01
:107EC00002C00E94293E2496CDBFDEBFCF91DF9134
:107ED0000895682F772767FD709580EA98E00E94E3
:107EE000EC2008959F92AF92BF92CF92DF92EF92D3
:107EF000FF920F931F93DF93CF93CDB7DEB7A99770
:107F0000CDBFDEBF0E94E5218AE090E061E671E42A
:107F10000E94D4210E9432228AE090E00E944320F5
:107F200097FD35C19090A80680EA98E040E855E2B8
:107F300060E070E028E030E000E010E0A1E0EA2E30
:107F4000F12CCC24DD240E94632097FD20C180EA1F
:107F500099E040E051EE60E070E028E030E00E94FF
:107F6000632097FD14C180E090E06CEE70E240EA7F
:107F700058E024E030E00E940A1A5C01009709F4FE
:107F800006C180ED97E020E233E0F9013197F1F787
:107F90000197D9F760E072EC81E090E040E02FEAD1
:107FA00031E203E011E2F0EAEF2EF9E0FF2E0E9449
:107FB000651597FDECC080EA99E040E052EC61E085
:107FC00070E028E030E000E010E0E1E0EE2EF12C7F
:107FD000CC24DD240E94632097FDD9C088EE93E075
:107FE00020E233E0F9013197F1F70197D9F788EDF5
:107FF00090E4B5010E94380D81EF90E4B5010E9434
:10800000410DC5016FE37DE240E050E00E945D1844
:10801000C50169E47DE240E050E00E945D18C501C1
:1080200063E57DE240E050E00E945D18C5016DE52A
:108030007DE240E050E00E945D18C50167E67DE208
:1080400040E050E00E945D18C50161E77DE240E03C
:1080500050E00E945D18C5016BE77DE240E050E012
:108060000E945D18C50165E87DE240E050E00E9495
:108070005D18C5016FED7DE240E050E00E945D18A3
:10808000C5016FE87DE240E050E00E945D18C50147
:1080900069E97DE240E050E00E945D18C50163EAB5
:1080A0007DE240E050E00E945D18C5016DEA7DE28E
:1080B00040E050E00E945D18C50167EB7DE240E0C2
:1080C00050E00E945D18C50161EC7DE240E050E0A7
:1080D0000E945D18C5016BEC7DE240E050E00E941B
:1080E0005D18C50165ED7DE240E050E00E945D183D
:1080F000C50165E37DE240E050E00E945D188FEF2E
:10810000981681F566E172E088EA90EC0E94EE151F
:1081100069837A838B839C8360E07FEF8FEF9FEF8F
:108120000E94EE156D837E838F8398878E01075F93
:108130001F4FC80162EC7CE20E9490458AE089A74B
:10814000C8016DEC7CE240E050E00E94DB14CE01FF
:108150000196BE016B5F7F4F40E050E020E030E0D1
:108160000E94290F80EA98E00E943C21892B51F05F
:1081700080EA98E060E070E00E949321682FC501DA
:108180000E946C1B0E943B110E94EC1EEBCF8FEFF4
:108190009FEFA996CDBFDEBFCF91DF911F910F91C9
:1081A000FF90EF90DF90CF90BF90AF909F90089599
:1081B00000D000D0EDB7FEB73196ADB7BEB711967F
:1081C0008D939C9312978BED9CE2828393836483BF
:1081D00075830E9483198DB79EB706968DBF9EBF8B
:1081E00008950F931F93182F092F6115710571F5CD
:1081F00000D00F92EDB7FEB73196ADB7BEB711966E
:108200008C9391838DEE9CE2828393830E948319E9
:108210008091B22E9091B32E0F900F900F900F90EF
:10822000009709F44BC00E94413E1092B22E10926A
:10823000B32E00D00F92EDB7FEB73196ADB7BEB7F3
:1082400011961C9301838FEF9CE230C0CB010E94FA
:10825000F51700D000D0EDB7FEB73196ADB7BEB779
:1082600011961C9301832FE03DE2228333838483A4
:1082700095830E9483198DB79EB706968DBF9EBFCA
:1082800080E590E00E94523E8093B22E9093B32EF0
:10829000892BA1F000D00F92EDB7FEB73196ADB7A4
:1082A000BEB711961C9301838FE19DE28283938375
:1082B0000E9483190F900F900F900F901F910F91B4
:1082C00008950E94911E0895629FD001739FF0014E
:1082D000829FE00DF11D649FE00DF11D929FF00D56
:1082E000839FF00D749FF00D659FF00D9927729F8D
:1082F000B00DE11DF91F639FB00DE11DF91FBD0118
:10830000CF0111240895991B79E004C0991F961795
:1083100008F0961B881F7A95C9F780950895AA1BC7
:10832000BB1B51E107C0AA1FBB1FA617B70710F060
:10833000A61BB70B881F991F5A95A9F78095909592
:10834000BC01CD01089597FB092E07260AD077FDC1
:1083500004D0E5DF06D000201AF4709561957F4FB8
:108360000895F6F7909581959F4F0895A1E21A2EF2
:10837000AA1BBB1BFD010DC0AA1FBB1FEE1FFF1FC9
:10838000A217B307E407F50720F0A21BB30BE40B19
:10839000F50B661F771F881F991F1A9469F7609560
:1083A0007095809590959B01AC01BD01CF0108951A
:1083B00097FB092E05260ED057FD04D0D7DF0AD033
:1083C000001C38F450954095309521953F4F4F4F04
:1083D0005F4F0895F6F790958095709561957F4F62
:1083E0008F4F9F4F08950F931F93CF93DF93689FF5
:1083F0008001699F100D789F100D1124C8010E9403
:108400000F42EC01009729F060E070E0A8010E94A3
:108410007545CE01DF91CF911F910F910895CF93B4
:10842000DF93BC018230910510F462E070E0A0910E
:10843000D12EB091D22EED0140E050E0E0E0F0E02E
:1084400021C0888199818617970769F48A819B8169
:10845000309719F08283938304C08093D12E909338
:10846000D22EFE0134C06817790738F44115510542
:1084700019F08417950708F4AC01FE018A819B81ED
:108480009C01E9012097E9F641155105A9F1CA01BE
:10849000861B970B049708F4BA01E0E0F0E02AC0CD
:1084A0008D919C91119784179507F9F464177507BE
:1084B00081F412968D919C911397309719F08283D5
:1084C000938304C08093D12E9093D22EFD013296D7
:1084D0004FC0CA01861B970BFD01E80FF91F61937E
:1084E000719302978D939C9343C0FD018281938188
:1084F0009C01D9011097A1F68091CF2E9091D02E9A
:10850000892B41F48091312D9091322D8093CF2E83
:108510009093D02E4091332D5091342D411551051B
:1085200041F44DB75EB780912F2D9091302D481BAF
:10853000590B2091CF2E3091D02E24173507B0F44F
:10854000CA01821B930B8617970780F0AB014E5F21
:108550005F4F8417950750F0420F531F4093CF2E63
:108560005093D02EF9016193719302C0E0E0F0E0E6
:10857000CF01DF91CF910895CF93DF93009709F456
:1085800050C0EC0122971A821B82A091D12EB0918B
:10859000D22E109709F140E050E0AC17BD0708F16A
:1085A000AA83BB83FE0121913191E20FF31FAE1725
:1085B000BF0779F48D919C911197280F391F2E5F79
:1085C0003F4F2883398312968D919C9113978A830C
:1085D0009B834115510571F4C093D12ED093D22EB7
:1085E00020C012968D919C911397AD01009711F0C8
:1085F000DC01D3CFFA01C283D38321913191E20F01
:10860000F31FCE17DF0769F488819981280F391F7E
:108610002E5F3F4FFA01208331838A819B818283C1
:108620009383DF91CF9108958F929F92AF92BF92E3
:10863000CF92DF92EF92FF920F931F93CF93DF932E
:108640008C01009729F4CB010E940F428C01BAC023
:108650009EEFE92E9FEFF92EE00EF11E5801A60EB7
:10866000B71EAE14BF0408F4ABC08EEF882E8FEF98
:10867000982E8A0C9B1CE7014881598146175707A1
:10868000B8F04530510508F49DC0CA01049786171B
:10869000970708F497C042505040461B570BF4010F
:1086A0004083518368837983C5010E94BC428AC09C
:1086B0006B01C41AD50AE091D12EF091D22EC0E000
:1086C000D0E0A0E0B0E042C0E815F905A1F52081B6
:1086D00031812C153D0578F1C90102968C159D0557
:1086E000A8F04E5F5F4F420F531FE7014883598345
:1086F00022813381109729F012962D933C93139782
:1087000061C02093D12E3093D22E5CC022503040D5
:108710002C193D0920833183109729F01296ED938F
:10872000FC93139704C0E093D12EF093D22EF7015F
:108730006083718347C080819181C817D90708F48D
:10874000EC01DF01828193819C01F901309709F0EE
:10875000BBCF400F511F8091CF2E9091D02E841708
:108760009507E9F4C617D707D0F42091332D30913F
:10877000342D2115310541F42DB73EB780912F2DB1
:108780009091302D281B390BA216B306C8F4A09285
:10879000CF2EB092D02EE7016883798313C0CB012E
:1087A0000E940F42EC01009759F0F701408151817E
:1087B000B8010E946C45C8010E94BC428E0102C0F3
:1087C00000E010E0C801DF91CF911F910F91FF9061
:1087D000EF90DF90CF90BF90AF909F908F900895D3
:1087E0002F923F925F926F927F928F929F92AF9261
:1087F000BF92CF92DF92EF92FF920F931F93CF938E
:10880000DF938C011B01EA016115710519F0FB0171
:1088100080839183209749F0CE010297839728F0B7
:1088200020E030E040E050E0F6C0F801A1908F0178
:108830008A2D90E00E944545892BB9F7FDE2AF16DD
:1088400031F4F801A1908F015524539407C0FBE245
:10885000AF1619F4F801A1908F015524209719F053
:10886000C031D105C1F4F0E3AF1679F4F80180818D
:10887000883711F0883549F4F801A1800E5F1F4F49
:10888000F2E05F2AC0E1D0E006C0209721F480E347
:10889000A816E9F427C0C830D10531F1C930D10597
:1088A00024F4C230D10531F50CC0CA30D10589F0AD
:1088B000C031D105F9F4C12CD12CE12CB8E0FB2E4C
:1088C00028C0C12CD12CE12CA0E4FA2E22C0CAE091
:1088D000D0E0FCECCF2EFCECDF2EFCECEF2EFCE02D
:1088E000FF2E17C0C8E0D0E0C12CD12CE12CE0E174
:1088F000FE2E0FC09E01442737FD4095542F60E0A7
:1089000070E080E090E80E94B641C901DA016C0194
:108910007D0120E030E040E050E060E03E0188244E
:1089200077FC8094982C70EDB72EBA0CE9E0EB152B
:1089300070F48A2D81548A3118F499ECB92E06C04E
:108940008A2D81568A3150F589EAB82EBA0C8B2DC2
:1089500090E08C179D0714F56F3FE1F0C216D30627
:10896000E406F506B0F0CA01B901A40193010E9422
:1089700064419B01AC012B0D311D411D511D213066
:10898000F0E03F07F0E04F07F0E85F0710F461E028
:1089900001C06FEFF801A1908F01C5CF2114310400
:1089A00081F0662331F001501040F1010083118302
:1089B00008C051FE1AC002501040F101008311831B
:1089C00014C067FF12C050FC05C02FEF3FEF4FEF00
:1089D0005FE704C020E030E040E050E882E290E051
:1089E0008093D32E9093D42E16C050FE08C050957D
:1089F0004095309521953F4F4F4F5F4F0CC057FF2B
:108A00000AC082E290E08093D32E9093D42E2FEF71
:108A10003FEF4FEF5FE7B901CA01DF91CF911F919F
:108A20000F91FF90EF90DF90CF90BF90AF909F900D
:108A30008F907F906F905F903F902F900895FC01F2
:108A400088279927E89421912032E9F3293010F002
:108A50002E30C8F32B3241F02D3239F4689404C023
:108A60000E94DB45820F911D219120532A30C0F3D3
:108A70001EF4909581959F4F0895803209F09111D1
:108A8000F4C580528F55E0F708959111EEC58032FC
:108A900019F089508550D0F70895911108958154A7
:108AA0008A5108F4805E855A0895FB01DC0102C0FA
:108AB00005900D9241505040D8F70895FC01059063
:108AC0000020E9F7809590958E0F9F1F08954EE83E
:108AD0005EE20E94B4450895FB01DC0102C00190F2
:108AE0000D9241505040D8F70895DC0101C06D93BC
:108AF00041505040E0F70895FB01DC010D9000204B
:108B0000E9F7119701900D920020E1F70895FB011C
:108B1000DC018D91019080190110D9F3990B089512
:108B2000FB01DC0101900D920020E1F70895FB01AB
:108B3000DC014150504030F08D910190801919F4C2
:108B40000020B9F7881B990B0895FB01DC01415007
:108B5000504048F001900D920020C9F701C01D92CD
:108B600041505040E0F70895FA01A191B08100977B
:108B700019F41097E1F0CD01DC01CD010D9000203A
:108B800011F4C00113C0FB012191222319F020151B
:108B9000D9F7F3CFFB012191201519F41E921196FC
:108BA00006C02223C1F70D900020A1F7D001FA01E1
:108BB000A193B08308957AE0979F902D879F802D91
:108BC000910D112408950F931F93DF93CF93CDB789
:108BD000DEB72E97CDBFDEBF0E891F89888D998D98
:108BE00097FF02C080E090E801978D839E83098300
:108BF0001A8386E08C839E01245E3F4FCE0101964E
:108C00006A8D7B8DA9010E9469464D815E8157FD69
:108C10000AC02F813885421753070CF49A01020FBE
:108C2000131FF80110822E96CDBFDEBFCF91DF91CA
:108C30001F910F910895DF93CF93CDB7DEB72E9795
:108C4000CDBFDEBF85E08C838C899D8989839A8323
:108C50009E01285E3F4FCE0101966E897F89A90152
:108C60000E94124A2E96CDBFDEBFCF91DF910895AC
:108C70000F931F93DF93CF93CDB7DEB72E97CDBF62
:108C8000DEBF8C0177FF02C060E070E86150704089
:108C90006D837E8309831A8386E08C83CE010196DF
:108CA000BA01A9010E9469462D813E8137FD09C0A4
:108CB000EF81F8852E173F070CF4F901E00FF11F43
:108CC00010822E96CDBFDEBFCF91DF911F910F9105
:108CD00008952F923F924F925F926F927F928F9260
:108CE0009F92AF92BF92CF92DF92EF92FF920F933B
:108CF0001F93DF93CF93CDB7DEB72B97CDBFDEBFEA
:108D00003C012B015A01FC0116821782838181FDEF
:108D100003C06FEF7FEFC6C19AE0892E1E01089451
:108D2000211C311CF3012381F20123FD859123FFD6
:108D300081912F01882309F4B2C1853239F423FDD2
:108D4000859123FF81912F01853229F490E0B301B1
:108D50000E949B4BE7CF982FFF24EE249924FFE13C
:108D6000FF15D0F09B3269F09C3228F4903259F014
:108D7000933291F40EC09D3249F0903369F441E092
:108D800024C052E0F52A84E0F82A28C098E0F92AA5
:108D900025C0E0E1FE2A22C0F7FC29C0892F8053BC
:108DA0008A3070F4F6FE05C0989C902C1124980E21
:108DB00015C0E89CE02C1124E80EF0E2FF2A0EC05A
:108DC0009E3229F4F6FC6BC140E4F42A07C09C36BD
:108DD00019F450E8F52A02C0983649F4F20123FD4F
:108DE000959123FF91912F01992309F0B8CF892FF5
:108DF0008554833018F08052833038F444E050E0DA
:108E0000A40EB51E5FE359830FC0933631F093373C
:108E100079F0933509F056C020C0F501808189832F
:108E200042E050E0A40EB51E610101E010E012C066
:108E3000F501C080D180F6FC03C06FEF7FEF02C068
:108E4000692D70E042E050E0A40EB51EC6010E94FC
:108E50004E4B8C015FE7F52214C0F501C080D18034
:108E6000F6FC03C06FEF7FEF02C0692D70E042E0B7
:108E700050E0A40EB51EC6010E94434B8C0150E881
:108E8000F52AF3FE07C01AC080E290E0B3010E9409
:108E90009B4BEA948E2D90E008171907A8F30EC09B
:108EA000F601F7FC8591F7FE81916F0190E0B30127
:108EB0000E949B4BE110EA940150104001151105EE
:108EC00079F7EAC0943611F0993669F5F7FE08C0D3
:108ED000F501208131814281538184E090E00AC014
:108EE000F501808191819C01442737FD4095542FE5
:108EF00082E090E0A80EB91E9FE6F92257FF09C054
:108F000050954095309521953F4F4F4F5F4FE0E88A
:108F1000FE2ACA01B901A1012AE030E00E94E14B1A
:108F2000D82ED21840C0953729F41F2D1F7E2AE075
:108F300030E01DC01F2D197F9F3661F0903720F45F
:108F4000983509F0ACC00FC0903739F0983709F068
:108F5000A6C004C028E030E00AC0106114FD14600F
:108F600020E130E004C014FD166020E132E017FF7C
:108F700008C0F501608171818281938144E050E0F5
:108F800008C0F50180819181BC0180E090E042E061
:108F900050E0A40EB51EA1010E94E14BD82ED218BC
:108FA0008FE7F82EF122F6FE0BC05EEFF522D91402
:108FB00038F4F4FE07C0F2FC05C08FEEF82202C0C0
:108FC0001D2D01C0192DF4FE0DC0FE01ED0DF11D8A
:108FD0008081803319F499EEF92208C01F5FF2FEF8
:108FE00005C003C08F2D867809F01F5F0F2DF3FC9D
:108FF00014C0F0FE0FC01E1510F09D2C0BC09D2C50
:109000009E0C911A1E2D06C080E290E0B3010E94D2
:109010009B4B1F5F1E15C0F304C01E1510F4E11A10
:1090200001C0EE2404FF0FC080E390E0B3010E9472
:109030009B4B02FF1DC001FD03C088E790E00EC0FE
:1090400088E590E00BC0802F867891F001FF02C088
:109050008BE201C080E2F7FC8DE290E0B3010E9458
:109060009B4B06C080E390E0B3010E949B4B9A9417
:10907000D914C0F3DA94F101ED0DF11D808190E077
:10908000B3010E949B4BDD20A9F706C080E290E06F
:10909000B3010E949B4BEA94EE20C1F743CEF3014B
:1090A00066817781CB012B96CDBFDEBFCF91DF915B
:1090B0001F910F91FF90EF90DF90CF90BF90AF90F6
:1090C0009F908F907F906F905F904F903F902F90E8
:1090D0000895FC0120FD08C023FD05C022FF02C049
:1090E00073836283518340830895EF92FF920F93BD
:1090F0001F9344FF02C033E011C046FF02C034E0BA
:109100000DC0DB01FC01AA0FBB1FEE1FFF1F109457
:10911000D1F76A0F7B1F8E1F9F1F31E0660F771FED
:10912000881F991F3150D1F77B018C01E20EF11C91
:10913000011D111DA8019701B701CA011F910F91CF
:10914000FF90EF9008950F931F93CF93DF938C01BF
:10915000C8010E94594BEC0197FD08C00E9445458B
:10916000892BB1F7CE01B8010E94C74BCE01DF9128
:10917000CF911F910F910895AF92BF92CF92DF923E
:10918000EF92FF920F931F93CF93DF93EC01C62EC4
:109190005A01122F0E94594BAC018B3219F08D32BB
:1091A00051F41068CA9409F46DC0CE010E94594B65
:1091B000AC0197FD67C06DEFD62ED1228D2D807347
:1091C00001F54033F1F4CA9409F447C0CE010E947E
:1091D000594BAC0197FD41C082E0D82A483711F0C5
:1091E000483559F480E4D82ACA94B9F1CE010E94D6
:1091F000594BAC0199232CF430C0D6FC02C080E15D
:10920000D82AEE24FF248701242F2053283088F009
:10921000D4FC09C02A3068F0D6FE05C02F7D822F0D
:109220008151863028F0CA01BE010E94C74B12C08E
:109230002750C801B7014D2D0E9475487B018C0154
:1092400082E0D82ACA9461F0CE010E94594BAC0149
:1092500097FFDACFD1FC04C015C0EE24FF248701AC
:10926000D7FE08C010950095F094E094E11CF11C25
:10927000011D111DC501B801A7012D2D0E946948CE
:1092800081E001C080E0DF91CF911F910F91FF90AD
:10929000EF90DF90CF90BF90AF9008956F927F9244
:1092A0008F929F92AF92BF92CF92DF92EF92FF92F6
:1092B0000F931F93DF93CF93CDB7DEB7A097CDBFAA
:1092C000DEBF6C01A62E8A017901FE01319680E293
:1092D000DF011D928A95E9F770E030E060E040E040
:1092E00050E04F01A1E0B0E0F6018381F70183FD7A
:1092F000259183FF21917F01222309F47EC02E3521
:1093000019F44115510569F1872F90E084179507ED
:1093100044F42D3551F12D3221F4332329F431E079
:1093200021C0332309F4622F322F832F869586952F
:109330008695F401E80FF11D832F87703D0102C06F
:10934000660C771C8A95E2F7208126292083361740
:1093500011F430E007C0361710F43F5FE6CF31500C
:10936000E4CF71E04F5F5F4FBFCF332319F08E81A1
:1093700080628E83772359F0FE0131969E012F5D26
:109380003F4F808180958193E217F307D1F7BB248B
:10939000B3944E010894811C911CC6010E94594B44
:1093A000AC0197FD22C0869586958695F401E80F5D
:1093B000F11D808190E09A012770307002C0959570
:1093C00087952A95E2F780FD05C0CA01B6010E9483
:1093D000C74B0BC00115110519F0D8014D938D0134
:1093E000AA94BB24AA20C9F602C0BB2031F40115FF
:1093F000110529F0F801108202C0EE24FF24C701F4
:10940000A096CDBFDEBFCF91DF911F910F91FF904E
:10941000EF90DF90CF90BF90AF909F908F907F9014
:109420006F9008956F927F928F929F92AF92BF92AA
:10943000CF92DF92EF92FF920F931F93CF93DF9320
:109440005C016B013A01FC01168217828824EAC094
:10945000812F90E00E944545892B21F0C5010E9493
:10946000A348E0C0153249F4F601F3FC6591F3FE20
:1094700061916F01653269F415E2C5010E94594B93
:1094800097FDDCC0181709F4CDC0B5010E94C74B89
:10949000DAC06A3219F0162F00E006C0F3FC15910D
:1094A000F3FE11916F0101E099240FC00260692D54
:1094B00070E080E090E040E20E947548962EF60150
:1094C000F3FC1591F3FE11916F01212F20532A30E7
:1094D00068F301FD03C099249A9403C0992009F40C
:1094E000B2C0183621F01C3699F4F6010BC0F60113
:1094F000F3FC6591F3FE6191683619F06F01162F48
:1095000007C008600460F3FC1591F3FE11916F0130
:10951000112309F498C085E09FE0612F70E00E945C
:10952000384B892B09F48FC0802F00FF03C0EE2435
:10953000FF2407C0F301E080F18022E030E0620EFA
:10954000731E1E3651F4F5014681578160E070E0CC
:10955000C701202F0E94694865C0133691F481FD30
:1095600002C099249394C5010E94594B97FD66C08F
:10957000E114F10419F0F70181937F019A9499F7AE
:109580004FC01B3559F4C501692DA70196010E94F2
:109590004E496C01009709F043C03DC0C5010E94CF
:1095A000A34897FD4BC01F3659F1103728F41436E5
:1095B00029F1193639F527C0133719F0153711F588
:1095C0001DC0C5010E94594BEC0197FD11C00E94BE
:1095D0004545892B29F0CE01B5010E94C74B08C033
:1095E000E114F10419F0F701C1937F019A9449F74E
:1095F000E114F104A9F0F701108212C0006203C067
:10960000006101C00064C501692DA701202F0E94DF
:10961000BC48882329F4F5018381807379F413C051
:1096200000FF8394F501F380F601F3FC1591F3FE3E
:1096300011916F01112309F00BCF05C0882019F497
:109640002FEF3FEF02C0282D30E0C901DF91CF910D
:109650001F910F91FF90EF90DF90CF90BF90AF9050
:109660009F908F907F906F900895992788270895F5
:10967000FC010590061621F00020D9F7C0010895DD
:109680003197CF010895FC010590615070400110A1
:10969000D8F7809590958E0F9F1F0895FC0161501B
:1096A000704001900110D8F7809590958E0F9F1F04
:1096B0000895CF93DF93EC014B8140FF1AC046FF22
:1096C0000AC04F7B4B838E819F8101968E839F833F
:1096D0008A81282F2BC042FF13C0E881F981808145
:1096E000282F332727FD30952115310529F44062B5
:1096F0004B832FEF3FEF1BC03196E883F98311C0F6
:10970000EA85FB85CE0119959C0197FF0AC09B81D4
:109710002F5F3F4F11F080E201C080E1892B8B83E6
:10972000E8CF8E819F8101968E839F8330E0C901AF
:10973000DF91CF9108950F931F93CF93DF938C0107
:10974000EB018B8181FF1BC082FF0DC02E813F8109
:109750008C819D812817390764F4E881F981019390
:10976000E883F98306C0E885F985802F1995892B50
:1097700031F48E819F8101968E839F8302C00FEF0B
:109780001FEFC801DF91CF911F910F9108959C01A8
:10979000FB01838180FF11C086FD0FC09FEF2F3F2B
:1097A000390759F0228380648F7D83838681978176
:1097B00001978683978330E002C02FEF3FEFC90106
:1097C0000895FA01AA27283051F1203181F1E89457
:1097D0006F936E7F6E5F7F4F8F4F9F4FAF4FB1E0A4
:1097E0003ED0B4E03CD0670F781F891F9A1FA11D9F
:1097F000680F791F8A1F911DA11D6A0F711D811DA0
:10980000911DA11D20D009F468943F912AE0269F64
:1098100011243019305D3193DEF6CF010895462FC3
:109820004770405D4193B3E00FD0C9F7F6CF462FA4
:109830004F70405D4A3318F0495D31FD405241930D
:1098400002D0A9F7EACFB4E0A695979587957795CA
:109850006795BA95C9F700976105710508959B0151
:10986000AC010A2E06945795479537952795BA95DA
:10987000C9F7620F731F841F951FA01D0895F894E8
:02988000FFCF18
:10988200200000252D3230732025730A0D0024009C
:10989200257320002573202D2068657864756D700E
:1098A200286C656E3D2564293A0A0D002530327810
:1098B2002000202020003A200020202025730A0DBD
:1098C20000082008000A0D00636F6D6D616E642050
:1098D2006E6F7420666F756E643A25730A0D0025EB
:1098E200630068656C70007072696E7420746869D8
:1098F2007320696E666F726D6174696F6E00257395
:10990200202D2068657864756D70286C656E3D2524
:1099120064293A0A0D0025303278200020202000E8
:109922003A200020202025730A0D007375636365B9
:10993200737300696E76616C696420706172616D27
:10994200657465727300756E6B6E6F776E206661FB
:10995200696C757265006F7574206F66206D656D38
:109962006F72792F62756666657273006E6F74200E
:10997200636F6E6E656374656400696E76616C69AF
:10998200642073746174650070617273696E67201C
:109992006572726F720070617468206E6F742066F7
:1099A2006F756E6400696E636F6D70617469626C6D
:1099B200652074797065006E6F207065726D6973D1
:1099C20073696F6E006F7065726174696F6E206E7D
:1099D2006F7420737570706F72746564006F757444
:1099E200206F662072616E67650062616420736930
:1099F2007A65007265747279206C617465720062B6
:109A02007573790064697361626C65640070726F6A
:109A1200746F636F6C206572726F720074696D652A
:109A22006F75740069676E6F7265640063616E635F
:109A3200656C65642062792072656D6F7465007370
:109A4200796E63206572726F720061626F72746503
:109A52006400616C726561647920696E207573655A
:109A6200002D2D2D20415353455254494F4E20462F
:109A720041494C4544202D2D2D0A0D002D412D200C
:109A820025733A25642025733A20300A0D002E2EC4
:109A92002F2E2E2F2E2E2F2E2E2F746F6F6C6B6962
:109AA200742F6F776C2F636F72652F6F776C5F65A2
:109AB20072722E6300756E6B6E6F776E002D2D2D98
:109AC20020415353455254494F4E204641494C453B
:109AD20044202D2D2D0A0D002D412D2025733A25D0
:109AE200642025733A202128746D6F2D3E666C61C7
:109AF2006773202620544D4F5F44454C45544544DE
:109B0200290A0D002E2E2F2E2E2F2E2E2F2E2E2FE7
:109B1200746F6F6C6B69742F6F776C2F636F7265E4
:109B22002F6F776C5F74696D65722E630045004E0E
:109B3200004F004D0053002D2D2D2041535345520F
:109B420054494F4E204641494C4544202D2D2D0A63
:109B52000D002D412D2025733A25642025733A20CE
:109B6200300A0D002E2E2F2E2E2F2E2E2F2E2E2F80
:109B7200746F6F6C6B69742F6F776C2F706F727468
:109B8200732F617672382F6F776C5F756172742EE6
:109B920063000076657273696F6E3A25642E2564E0
:109BA2002E25642028636F64653A2564290A0D0016
:109BB200636F6E6E5F636220736F636B69643A25D5
:109BC2006420636F6E6E65637465643A25640A0D82
:109BD20000657272006F6B002573202564202825B2
:109BE2007329200076657273696F6E3A25642E259B
:109BF200642E25642028636F64653A2564292062F7
:109C020075696C643A25730A0D002573202564205A
:109C1200282573290A0D0075736167653A20676507
:109C2200745F686F737462796E616D65203C646EF7
:109C3200736E616D653E0A0D006C6F6F6B75705FC0
:109C420063623A20686F7374206E6F7420666F755A
:109C52006E640A0D006C6F6F6B75705F63622069D2
:109C6200703A25730A0D00706565723A25730A0D04
:109C72000075736167653A206765745F7065657228
:109C820061646472203C736F636B69643E0A0D0009
:109C920073656E64696E67202564206279746573EA
:109CA20020746F2025733A25640A0D0077726F7451
:109CB200653A25642072656D61696E3A25640A0D04
:109CC2000075736167653A2073656E64746F203C3A
:109CD200736F636B69643E203C69703E203C706F19
:109CE20072743E203C64617461202E2E2E3E0A0D59
:109CF2000073656E64696E672025642062797465FD
:109D0200730A0D0075736167653A2073656E64208E
:109D12003C736F636B69643E203C64617461202E06
:109D22002E2E3E0A0D0075736167653A20636C6FD3
:109D32007365203C736F636B69643E0A0D00757333
:109D42006167653A20636F6E6E656374203C736F62
:109D5200636B69643E203C69703E203C706F727494
:109D62003E0A0D0075736167653A206C697374650C
:109D72006E203C736F636B69643E205B6261636B50
:109D82006C6F675D0A0D006C697374656E5F636268
:109D920020736F636B69643A25642C206163636589
:109DA2007074696E67202E2E2E200028636F6E6EEF
:109DB200656374696F6E206C6F737429000072653D
:109DC20063765F636220736F636B69643A25642014
:109DD2006C656E3A25642025730A0D005258007591
:109DE200736167653A2062696E64203C736F636BCE
:109DF20069643E203C69703E203C706F72743E0A7A
:109E02000D0073747265616D00646772616D00723A
:109E120061770075736167653A20736F636B657470
:109E2200203C73747265616D7C646772616D7C72D3
:109E320061773E205B70726F746F636F6C5D0A0DA9
:109E42000025732025642028656E61626C65643A82
:109E52002564290A0D0075736167653A207365747C
:109E62005F64686370203C307C313E0A0D002573CC
:109E720020256420280069703A257320006D6173E3
:109E82006B3A2573200067773A25732000646E735E
:109E92003A2573290A0D0075736167653A20736567
:109EA200745F697061646472203C69703E205B6D0E
:109EB20061736B5D205B67775D205B646E735D0A27
:109EC2000D004E2F41002573202564202825732084
:109ED200253032783A253032783A253032783A25B0
:109EE2003032783A253032783A25303278290A0DE4
:109EF2000025732025642028253032783A25303217
:109F0200783A253032783A253032783A253032782C
:109F12003A25303278290A0D0075736167653A2057
:109F22006C696E6B7570205B737369645D205B6B2B
:109F320065795D205B7765705D0A0D006C696E6BFB
:109F4200757000776C705F6C696E6B7570287373D7
:109F520069642C206B65792C2077657029006C6907
:109F62006E6B646F776E00776C705F6C696E6B649A
:109F72006F776E2829006765745F68776164647221
:109F820000776C705F6765745F68776164647228DC
:109F920029006765745F6E6574776F726B00776C0A
:109FA200705F6765745F6E6574776F726B282900E6
:109FB2007365745F69706164647200776C705F735B
:109FC20065745F6970616464722869702C206D61C8
:109FD200736B2C2067772C20646E7329006765747D
:109FE2005F69706164647200776C705F6765745F4B
:109FF2006970616464722829007365745F646863C0
:10A002007000776C705F7365745F64686370286555
:10A012006E61626C6529006765745F6468637000D5
:10A02200776C705F6765745F64686370282900737A
:10A032006F636B657400776C705F736F636B6574CD
:10A0420028747970652C2070726F746F29006269B0
:10A052006E6400776C705F62696E6428736F636B05
:10A062002C2069702C20706F727429006C697374D3
:10A07200656E00776C705F6C697374656E28736FC0
:10A08200636B69642C206261636B6C6F6729006388
:10A092006F6E6E65637400776C705F636F6E6E6572
:10A0A200637428736F636B69642C2069702C207051
:10A0B2006F72742900636C6F736500776C705F63F5
:10A0C2006C6F736528736F636B6964290073656EC7
:10A0D2006400776C705F73656E6428736F636B697D
:10A0E200642C2064617461290073656E64746F006E
:10A0F200776C705F73656E64746F28736F636B69DE
:10A10200642C20646174612C2069702C20706F7241
:10A112007429006765745F706565726164647200BA
:10A12200776C705F6765745F706565726164647295
:10A1320028736F636B696429006765745F686F7366
:10A142007462796E616D6500776C705F6765745FCC
:10A15200686F737462796E616D6528646E736E6187
:10A162006D6529006765745F66775F7665727369EE
:10A172006F6E00776C705F6765745F66775F766598
:10A182007273696F6E28636F64652C206275696CE7
:10A192006429006765745F76657273696F6E00701B
:10A1A20072696E742076657273696F6E000A0D00B3
:10A1B20074746370206572723A25642028257329AD
:10A1C2000A0D0074746370206F6B3A20256420625C
:10A1D200797465732070726F636573736564206947
:10A1E2006E202564206D732C2025642E2564204B5F
:10A1F200422F730A0D0074746370206F6B3A20252E
:10A20200642062797465732070726F63657373651D
:10A212006420696E2030206D730A0D002E002D2DF2
:10A222002D20415353455254494F4E204641494CEB
:10A232004544202D2D2D0A0D002D412D2025733A48
:10A2420025642025733A20707269762D3E73656EFF
:10A25200640A0D002E2E2F2E2E2F776C705F7474D1
:10A2620063702E63002D412D2025733A256420252D
:10A27200733A20706F73203D3D20707269762D3ED7
:10A282006275666C656E0A0D002D70002D6E002DD4
:10A292006C002D74002D7200257320256420282562
:10A2A20073290A0D00657272007474637020636F03
:10A2B2006E6E6563742025733A2564206E6275663E
:10A2C2003A2564206275666C656E3A256420736F68
:10A2D200636B69643A25640A0D0074746370206CC0
:10A2E200697374656E20706F72743A2564206275AA
:10A2F200666C656E3A2564206C736F636B69643AB1
:10A3020025640A0D0075736167653A207474637081
:10A31200205B2D7472706E6C5D0A0D007474637034
:10A322000074746370207468726F756768707574F6
:10A332002074657374006661696C656420746F20B3
:10A34200676574206E74702074696D653A25732890
:10A352002564290A0D006E74702074696D653A20B7
:10A36200253034642D253032642D25303264202589
:10A372003032643A253032643A253032640A0D00B4
:10A38200657272006F6B0025732025642028257387
:10A39200290A0D0075736167653A206E7470203C5E
:10A3A2006E74702D7365727665723E0A0D006E745E
:10A3B2007000676574207365727665722074696DCA
:10A3C200652066726F6D206E7470002D2D2D202514
:10A3D200732070696E672073746174697374696342
:10A3E20073202D2D2D0A0D002564207061636B658D
:10A3F2007473207472616E736D69747465642C2059
:10A4020025642072656365697665640A0D002564BA
:10A412002062797465732066726F6D2025733A200D
:10A4220069636D705F7365713D25640A0D00256473
:10A432002062797465732066726F6D2025733A20ED
:10A4420069636D705F7365713D2564204465737443
:10A45200696E6174696F6E20486F737420556E72F5
:10A462006561636861626C650A0D0025642062792A
:10A472007465732066726F6D2025733A2069636D6F
:10A48200705F7365713D256420547970653A256467
:10A492000A0D002D63002D7300657272006F6B0050
:10A4A200257320256420282573290A0D0075736100
:10A4B20067653A2070696E67205B2D63203C636F8D
:10A4C200756E743E5D205B2D73203C73697A653E28
:10A4D2005D203C69703E0A0D0070696E67004E2F68
:10A4E2004100253032783A253032783A25303278B8
:10A4F2003A253032783A253032783A2530327800AF
:10A5020025642043002F002F3F002F696E64657879
:10A512002E68746D6C3F00746F67676C653D4C45C7
:10A52200442564002F696E6465782E68746D6C0032
:10A532002F6C6F676F2E676966000D0A00474554DE
:10A5420020006864776972656C657373006864776C
:10A552006972656C657373313233006C696E6B5F5F
:10A562006362206C696E6B3A25640A0D0061646453
:10A57200725F63622069703A6E6F6E650A0D0068E1
:10A58200747470642073746F707065640A0D006176
:10A592006464725F63622069703A25730A0D006811
:10A5A2007474706420737461727465640A0D00209F
:10A5B20000D52E00006220CC19672000000000BCEC
:10A5C200262C2EC32600000000DE26F02DE72600F2
:10A5D200000000F626A42D0127000000001227FE2D
:10A5E2002C1E27000000003027412C3B27000000D2
:10A5F200005D278D2B6827000000007927172B822A
:10A6020027000000009727DA2AA02700000000AFE9
:10A6120027222AB62700000000CE277229D327005E
:10A62200000000EC27FD27F327000000000F284D53
:10A63200271728000000003528D7263B28000000F5
:10A64200004D28DC255228000000006928AB247048
:10A65200280000000093281324A02800000000B95D
:10A66200287D23C82800000000E428F222F32800F5
:10A6720000000013299A221F29000000009C2A5A78
:10A6820032A12A000000002E2B4837322B00000096
:10A6920000592C7D39592C0000000000000000FFF9
:10A6A200FFFFFF6F776C5F6572726F72006F776C7E
:10A6B200746D725F64656C746D6F006F776C756139
:10A6C20072745F70617269747900636F6E6E5F633A
:10A6D200620073656E646275660000001F003B00D5
:10A6E2005A0078009700B500D400F3001101300140
:10A6F2004E016D0100001F003C005B0079009800D4
:0EA70200B600D500F400120131014F016E01C6
:00000001FF
